:100000000C942A000C9446240C9436240C9447003B
:100010000C9447000C94B6230C9447000C94E923ED
:100020000C9426240C9416240C9466230C94EE2233
:100030000C9447000C946B250C9417250C944700E6
:100040000C9447000C9447000C9447000C94470014
:100050000C94470011241FBECFE5D8E0DEBFCDBF12
:1000600011E0A0E6B0E0E6E6FAE702C005900D92E6
:10007000A437B107D9F714E0A4E7B1E001C01D929D
:10008000A033B107E1F70E9449000C94323D0C9473
:100090000000AF92BF92CF92DF92EF92FF920F9348
:1000A0001F93CF93DF93CDB7DEB7AE970FB6F8941B
:1000B000DEBF0FBECDBFEAE3F0E01082E7E3F0E081
:1000C0001082E4E3F0E01082E1E3F0E08FEF808360
:1000D000A1E3B0E0E1E3F0E0808180688C93A1E3EC
:1000E000B0E0E1E3F0E0808180648C93E2E3F0E053
:1000F00080818F778083E2E3F0E080818064808379
:100100000E94BB220E949A230E94C9240E94E824D4
:10011000A7E3B0E0E7E3F0E0808181608C93A7E3A0
:10012000B0E0E7E3F0E0808184608C93A7E3B0E087
:10013000E7E3F0E0808182608C93A7E3B0E0E7E33F
:10014000F0E0808188608C93A7E3B0E0E7E3F0E023
:10015000808180618C93A1E3B0E0E1E3F0E08081F5
:10016000877F8C93A1E3B0E0E1E3F0E080818B7FB7
:100170008C93AAE3B0E0EAE3F0E0808180628C93A4
:10018000AAE3B0E0EAE3F0E0808180618C93A1E330
:10019000B0E0E1E3F0E0808180618C93A1E3B0E026
:1001A000E1E3F0E0808180628C93E2E3F0E0808123
:1001B0008F7E8083E8E3F0E080818E7F8083E8E3B8
:1001C000F0E080818D7F8083E8E3F0E080818B7FA9
:1001D0008083E8E3F0E08081877F8083E8E3F0E0DC
:1001E00080818F7E8083A4E3B0E0E4E3F0E080814F
:1001F00081608C93E5E3F0E080818E7F8083A4E3CF
:10020000B0E0E4E3F0E0808182608C93E5E3F0E02D
:1002100080818D7F8083A4E3B0E0E4E3F0E080811F
:1002200084608C93E5E3F0E080818B7F8083A4E39E
:10023000B0E0E4E3F0E0808188608C93E5E3F0E0F7
:100240008081877F8083A4E3B0E0E4E3F0E08081F5
:1002500080618C93A4E3B0E0E4E3F0E0808180620D
:100260008C93A4E3B0E0E4E3F0E0808180648C93BD
:10027000A4E3B0E0E4E3F0E0808180688C93E5E300
:10028000F0E080818F7E8083E5E3F0E080818F7DE8
:100290008083E5E3F0E080818F7B8083E5E3F0E01D
:1002A0008081806880838CE291E00E94E527DC01F8
:1002B000CB018093930090939400A0939500B0930A
:1002C000960080E391E00E94E527DC01CB0180935A
:1002D000970090939800A0939900B0939A000E9481
:1002E000A81B0E942A177894A1E3B0E0E1E3F0E0B4
:1002F000808182608C93A1E3B0E0E1E3F0E0808153
:100300008E7F8C938AEA0E94F82581E00E94F8256E
:1003100080E00E94F82585E50E94F82582E0809320
:100320007B018091930090919400A0919500B091F1
:1003300096001EA62DEC3CEC4CEC5EE3BC01CD011E
:100340000E94FE3B88230CF002C001E00EA781E072
:100350001EA581278823D9F4809193009091940061
:10036000A0919500B09196001DA62FE832EC45EFC4
:100370005CE3BC01CD010E94013C18160CF002C0E8
:1003800021E02DA781E03DA583278823C1F087E1E7
:100390009FE9A2E0BDE38093930090939400A09323
:1003A0009500B093960080E090ECACE1B1E48093CE
:1003B000970090939800A0939900B0939A004AE018
:1003C00050E060E070E082E00E94B91D109276017A
:1003D0001092770110927801109279011092EE013B
:1003E0001092EF011092F0011092F1011092EA01C7
:1003F0001092EB011092EC011092ED011092E201CB
:10040000A5E3B0E0E5E3F0E08081881F8827881F3E
:100410008170982F990F990F8C918B7F892B8C93DA
:10042000A5E3B0E0E5E3F0E08081829586958695CE
:10043000837081708170982F990F8C918D7F892B9B
:100440008C93A8958091EB009091EC00A091ED0029
:10045000B091EE00813863EC960769ECA60761E085
:10046000B60710F00E94EA1B80911E0290911F02B5
:10047000A0912002B09121020097A105B10509F0D9
:10048000CBC0E0E3F0E080818870882351F42091B4
:100490009701309198018091880099272817390792
:1004A00044F58091DC019091DD0101969093DD018E
:1004B0008093DC018091DC019091DD0178E8883B3C
:1004C000970708F4A9C08091DB01882309F0A4C034
:1004D00040E050E060E070E081E00E94B91D81E002
:1004E0008093DB0188EB98E89093DD018093DC0139
:1004F00093C08091DC019091DD0101979093DD0123
:100500008093DC018091DC019091DD018B309105BD
:1005100008F082C08091DB01813009F07DC010922B
:10052000DB018AE090E09093DD018093DC01809113
:10053000D5018E31F1F58091EB009091EC00A09106
:10054000ED00B091EE0024E630E040E050E0BC0168
:10055000CD010E94FC3CDA01C9019C01AD018091F2
:10056000700090917100AA27BB27280F391F4A1FDE
:100570005B1F8091700090917100AA27BB27280F04
:10058000391F4A1F5B1F8091700090917100AA274C
:10059000BB27820F931FA41FB51F4496A11DB11D39
:1005A0008093EE019093EF01A093F001B093F101DD
:1005B00033C08091EB009091EC00A091ED00B091E0
:1005C000EE0024E630E040E050E0BC01CD010E94A6
:1005D000FC3CDA01C9019C01AD0180917000909151
:1005E0007100AA27BB27280F391F4A1F5B1F809164
:1005F000700090917100AA27BB27820F931FA41F40
:10060000B51F4496A11DB11D8093EE019093EF019B
:10061000A093F001B093F1010E94E0218091D501F7
:10062000E82EFF24FCA6EBA60BA51CA50E31110598
:1006300011F40C949C0C2BA53CA52F3131053CF5F5
:100640006BA57CA56A30710509F44BC58BA59CA5EB
:100650008B30910574F4EBA4FCA4E114F10409F4CB
:1006600049C00BA51CA50930110509F447C10C941C
:1006700063132BA53CA52331310509F4C3C76BA532
:100680007CA56431710509F4F0C70C9463138BA544
:100690009CA58832910511F40C94E9100BA51CA5BA
:1006A0000932110584F42BA53CA52F31310511F435
:1006B0000C944D0E6BA57CA56032710511F40C9461
:1006C000BC0E0C9463138BA59CA58D33910511F47E
:1006D0000C9422120BA51CA50336110511F40C94E1
:1006E00032132BA53CA52C33310511F40C94A71122
:1006F0000C9463131092E3011092E401E5E3F0E03F
:1007000080818E7F8083E5E3F0E080818D7F808330
:100710008091E201882351F48091E7019091E801F2
:10072000009721F01092E8011092E7018091EB0010
:100730009091EC00A091ED00B091EE00893833E18A
:10074000930730E0A30730E0B30710F40C9465136F
:100750001092E6011092E501809182009091830051
:10076000AC0160E070E080E00E94B91D209187013B
:10077000309188018091780099272817390724F053
:1007800088E28093D501B0C080918B0190918C015B
:10079000883C91050CF46EC083E18093D5018FE015
:1007A00090E09093D8018093D7011092D901809165
:1007B000EE019091EF01A091F001B091F10100974D
:1007C000A105B10509F090C08091EA019091EB017B
:1007D000A091EC01B091ED010097A105B10509F0E0
:1007E00083C0209170003091710080916E009091D3
:1007F0006F00820F931FAA27BB278093EB00909373
:10080000EC00A093ED00B093EE008091EB0090918E
:10081000EC00A091ED00B091EE002AE030E040E065
:1008200050E0BC01CD010E94B63CDC01CB018093BD
:10083000EB009093EC00A093ED00B093EE0080915C
:10084000EB009091EC00A091ED00B091EE002AE059
:1008500030E040E050E0BC01CD010E94B63CDC013C
:10086000CB018093EB009093EC00A093ED00B0934C
:10087000EE003AC080918B0190918C0187399105EF
:10088000D4F089E08093D5011092D8011092D7015D
:100890001092EA011092EB011092EC011092ED011E
:1008A0001092EE011092EF011092F0011092F101FE
:1008B0001092D90119C089E08093D5011092D80116
:1008C0001092D7011092EA011092EB011092EC0104
:1008D0001092ED011092EE011092EF011092F001D2
:1008E0001092F1011092D9011092EA011092EB01DD
:1008F0001092EC011092ED010C94651310927601A8
:100900001092770110927801109279018091220261
:1009100090912302A0912402B09125022091EB0036
:100920003091EC004091ED005091EE0028513C4F89
:100930004F4F5F4F82179307A407B50738F448EE6F
:1009400053E060E070E082E00E94B91D80912602D1
:1009500090912702A0912802B09129020097A10549
:10096000B10509F07AC08091EA019091EB01A09164
:10097000EC01B091ED010097A105B10509F06DC042
:100980000E942A17809177008093E301809177007D
:100990008093E4018091740190917501AC0160E055
:1009A00070E083E00E94B91D8091E2018F5F809327
:1009B000E2018091D7019091D8019093D801809362
:1009C000D7018091E201823088F080916800909197
:1009D000690023E030E0B9010E94D53CCB01AC01B5
:1009E00060E070E081E00E94B91D0AC0809168005B
:1009F00090916900AC0160E070E081E00E94B91D57
:100A00008091EA019091EB01A091EC01B091ED0190
:100A10000196A11DB11D8093EA019093EB01A09373
:100A2000EC01B093ED018091EB009091EC00A0916E
:100A3000ED00B091EE0024E630E040E050E0BC0173
:100A4000CD010E94FC3CDA01C9018093EE01909334
:100A5000EF01A093F001B093F101809126029091F3
:100A60002702A0912802B09129020097A105B105A3
:100A700009F06FC08091EA019091EB01A091EC0127
:100A8000B091ED0181309105A105B10509F061C07A
:100A900080911E0290911F02A0912002B09121022C
:100AA0000097A105B10509F054C0809166009091AE
:100AB0006700AC0160E070E083E00E94B91D8091A6
:100AC000D7019091D8019093D8018093D70140EB42
:100AD00054E060E070E084E00E94B91D81E090E0A5
:100AE0009093E6018093E5018091EA019091EB01FA
:100AF000A091EC01B091ED010196A11DB11D809373
:100B0000EA019093EB01A093EC01B093ED01809189
:100B1000EB009091EC00A091ED00B091EE0024E686
:100B200030E040E050E0BC01CD010E94FC3CDA0125
:100B3000C9018093EE019093EF01A093F001B0936F
:100B4000F101809177008093E30180917700809399
:100B5000E40180912A0290912B02A0912C02B09185
:100B60002D022091EB003091EC004091ED0050916E
:100B7000EE0028513C4F4F4F5F4F82179307A40759
:100B8000B507B8F48091E5019091E60185309105B3
:100B900080F440EB54E060E070E084E00E94B91D16
:100BA0008091E5019091E60101969093E601809392
:100BB000E5018091260290912702A0912802B09130
:100BC00029020097A105B10539F58091EA019091BC
:100BD000EB01A091EC01B091ED010097A105B105E9
:100BE000D9F080918B0190918C01883C9105A4F4FF
:100BF0008091820090918300AC0160E070E080E021
:100C00000E94B91D8091660090916700AC0162E37B
:100C100070E083E00E94B91D80918B0190918C015E
:100C20009C0180917400909175008217930708F5DC
:100C300080912A0290912B02A0912C02B0912D025A
:100C40000097A105B10569F440E157E260E070E06A
:100C500084E00E94B91D8AE090E09093E6018093C1
:100C6000E501809176008093E30180917600809386
:100C7000E4018091EA019091EB01A091EC01B09127
:100C8000ED0182309105A105B10508F4FEC0809107
:100C9000EA019091EB01A091EC01B091ED01883057
:100CA0009105A105B10508F0F0C080911E02909158
:100CB0001F02A0912002B09121020097A105B10569
:100CC00009F0E3C080918B0190918C018C0180919F
:100CD000EA019091EB01A091EC01B091ED0129E1C5
:100CE00030E040E050E0BC01CD010E94B63CDC01A8
:100CF000CB019C018091740090917500820F931F2D
:100D0000C2978017910708F0C0C08091EB009091C6
:100D1000EC00A091ED00B091EE0024E630E040E060
:100D200050E0BC01CD010E94FC3CDA01C9019C01EC
:100D3000AD018091EE019091EF01A091F001B09191
:100D4000F10179018A01E81AF90A0A0B1B0BD80193
:100D5000C70183339105A105B10508F496C08091C0
:100D6000EB009091EC00A091ED00B091EE0024E634
:100D700030E040E050E0BC01CD010E94FC3CDA01D3
:100D8000C9019C01AD018091EE019091EF01A0910C
:100D9000F001B091F10182179307A407B50708F09D
:100DA00074C080919701909198019C0180919B0063
:100DB00090919C002817390708F067C040E157E27E
:100DC00060E070E084E00E94B91D80916A0090911B
:100DD0006B0020918D0030918E00AC01B90181E053
:100DE0000E94B91D8091EA019091EB01A091EC0164
:100DF000B091ED010196A11DB11D8093EA01909380
:100E0000EB01A093EC01B093ED018091EB00909188
:100E1000EC00A091ED00B091EE0024E630E040E05F
:100E200050E0BC01CD010E94FC3CDA01C9019C01EB
:100E3000AD0180918D0090918E00AA27BB27280FCD
:100E4000391F4A1F5B1F80916A0090916B00AA278F
:100E5000BB27820F931FA41FB51F8093EE019093B1
:100E6000EF01A093F001B093F10180918600909181
:100E7000870090938E0080938D0080917600809300
:100E8000E301809176008093E4018091EA019091E2
:100E9000EB01A091EC01B091ED0188309105A10525
:100EA000B10508F4ABC080911E0290911F02A09181
:100EB0002002B09121020097A105B10509F09EC062
:100EC00080918B0190918C019C018091890090917F
:100ED0008A008217930708F040C080919701909193
:100EE00098019C0180919B0090919C0028173907E4
:100EF000A0F54AE050E060E070E082E00E94B91D99
:100F00001092EA011092EB011092EC011092ED01A7
:100F10008AE08093D50140ED57E060E070E082E028
:100F20000E94B91D8091EB009091EC00A091ED0022
:100F3000B091EE0024E630E040E050E0BC01CD018D
:100F40000E94FC3CDA01C9018093EE019093EF010D
:100F5000A093F001B093F10151C08091EB0090910A
:100F6000EC00A091ED00B091EE0024E630E040E00E
:100F700050E0BC01CD010E94FC3CDA01C9019C019A
:100F8000AD018091EE019091EF01A091F001B0913F
:100F9000F10180559B4FAF4FBF4F82179307A407B6
:100FA000B50760F54AE050E060E070E082E00E9442
:100FB000B91D1092EA011092EB011092EC0110920F
:100FC000ED018AE08093D5018091EB009091EC00D7
:100FD000A091ED00B091EE0024E630E040E050E05A
:100FE000BC01CD010E94FC3CDA01C9018093EE01F5
:100FF0009093EF01A093F001B093F101809126024C
:1010000090912702A0912802B09129020097A10592
:10101000B10571F080918B0190918C01893C910513
:101020003CF040E050E060E070E083E00E94B91DD9
:101030008091EA019091EB01A091EC01B091ED015A
:1010400082309105A105B10550F180912A0290915D
:101050002B02A0912C02B0912D020097A105B105A1
:10106000F1F48091E5019091E60185309105B8F0A9
:1010700080918B0190918C018436910584F480914C
:10108000E201833048F41092D50181E090E0909322
:10109000E8018093E70103C083E68093D5012091A6
:1010A0008701309188018091780099270A96281746
:1010B000390714F40C94651388E28093D50180916C
:1010C0008B0190918C019093DF018093DE018091E0
:1010D000DE019091DF019093E1018093E0010C9497
:1010E0006513109276011092770110927801109298
:1010F0007901A8951092E8011092E7011092E2019F
:101100008091260290912702A0912802B091290295
:101110000097A105B10571F080918B0190918C0130
:10112000893C91053CF040E050E060E070E083E0F5
:101130000E94B91D8091220290912302A091240265
:10114000B09125022091EB003091EC004091ED0030
:101150005091EE0028513C4F4F4F5F4F821793073D
:10116000A407B50738F440ED57E060E070E082E096
:101170000E94B91D80911A0290911B02A0911C023D
:10118000B0911D020097A105B105C9F48091EA0153
:101190009091EB01A091EC01B091ED010097A105B8
:1011A000B10569F0809182009091830020918400C4
:1011B00030918500AC01B90180E00E94B91D809199
:1011C00076008093E401809176008093E301209182
:1011D0002A0230912B0240912C0250912D028091D5
:1011E000EB009091EC00A091ED00B091EE008851E1
:1011F0009C4FAF4FBF4F281739074A075B0738F49A
:1012000048EE53E060E070E084E00E94B91D8091F8
:101210001E0290911F02A0912002B091210200971E
:10122000A105B10509F0D4C08091EA019091EB01CC
:10123000A091EC01B091ED010097A105B10509F075
:10124000C7C08091EB009091EC00A091ED00B091AF
:10125000EE0024E630E040E050E0BC01CD010E9409
:10126000FC3CDA01C9019C01AD018091EE01909135
:10127000EF01A091F001B091F10182179307A4074B
:10128000B50708F0A5C08091EB009091EC00A0910B
:10129000ED00B091EE0024E630E040E050E0BC010B
:1012A000CD010E94FC3CDA01C9019C01AD01809195
:1012B000EE019091EF01A091F001B091F101281B96
:1012C000390B4A0B5B0B80918B0090918C00AA2705
:1012D000BB2782179307A407B50708F079C0809150
:1012E0008B0190918C015C01CC24B7FCC094DC2C68
:1012F00080917200909173007C01002711278091EA
:101300008F009927AA27BB272091EA013091EB0192
:101310004091EC015091ED01BC01CD010E94B63C21
:10132000DC01CB018E0D9F1DA01FB11F8A159B05EF
:10133000AC05BD0508F02CC18091970190919801F2
:101340009C0180919B0090919C002817390708F020
:101350001FC120916E0030916F00C901880F991F45
:10136000820F931F96958795AC0160E070E081E055
:101370000E94B91D8091EA019091EB01A091EC01CE
:10138000B091ED010196A11DB11D8093EA019093EA
:10139000EB01A093EC01B093ED018091EB009091F3
:1013A000EC00A091ED00B091EE0024E630E040E0CA
:1013B00050E0BC01CD010E94FC3CDA01C9018093E0
:1013C000EE019093EF01A093F001B093F101E0C022
:1013D00080911E0290911F02A0912002B0912102E3
:1013E0000097A105B10509F0D3C08091EA01909161
:1013F000EB01A091EC01B091ED010097A105B105C1
:1014000009F4C6C08091EB009091EC00A091ED0032
:10141000B091EE0024E630E040E050E0BC01CD01A8
:101420000E94FC3CDA01C9019C01AD018091EE01F2
:101430009091EF01A091F001B091F1018217930713
:10144000A407B50708F0A4C08091EB009091EC00D0
:10145000A091ED00B091EE0024E630E040E050E0D5
:10146000BC01CD010E94FC3CDA01C9019C01AD0127
:101470008091EE019091EF01A091F001B091F10106
:10148000BA01A901481B590B6A0B7B0B2091700014
:101490003091710080916E0090916F00820F931FC8
:1014A000AA27BB2784179507A607B70708F070C0BF
:1014B00080918B0190918C015C01CC24B7FCC0948D
:1014C000DC2C80917200909173007C010027112721
:1014D00080918F009927AA27BB272091EA0130919C
:1014E000EB014091EC015091ED01BC01CD010E9456
:1014F000B63CDC01CB018E0D9F1DA01FB11F8A15CC
:101500009B05AC05BD0508F043C080919701909103
:1015100098019C0180919B0090919C0028173907AD
:10152000B8F580916E0090916F00AC0160E070E0C2
:1015300081E00E94B91D8091EA019091EB01A09198
:10154000EC01B091ED010196A11DB11D8093EA015E
:101550009093EB01A093EC01B093ED018091EB002F
:101560009091EC00A091ED00B091EE0024E630E007
:1015700040E050E0BC01CD010E94FC3CDA01C90111
:101580008093EE019093EF01A093F001B093F101ED
:101590008091EA019091EB01A091EC01B091ED01F5
:1015A00086309105A105B10518F083E18093D5013E
:1015B00080918B0190918C018436910514F41092E6
:1015C000D501209187013091880180917800992779
:1015D0002817390714F40C9465138EE18093D50114
:1015E00080918B0190918C019093DF018093DE01BB
:1015F0008091DE019091DF019093E1018093E00101
:101600000C94651384E18093D5011092EA01109245
:10161000EB011092EC011092ED010E942A17E5E314
:10162000F0E0808181608083E5E3F0E0808182608A
:1016300080831092D8011092D7011092E20180911C
:10164000EB009091EC00A091ED00B091EE0088517C
:101650009C4FAF4FBF4F8093760190937701A0933B
:101660007801B09379010C94651380917600809392
:10167000E401809176008093E30180911A029091B9
:101680001B02A0911C02B0911D020097A105B1059B
:1016900069F48091820090918300209184003091C0
:1016A0008500AC01B90180E00E94B91D80912A0239
:1016B00090912B02A0912C02B0912D022091EB0071
:1016C0003091EC004091ED005091EE0028513C4FDC
:1016D0004F4F5F4F82179307A407B50738F440EBCD
:1016E00054E060E070E084E00E94B91D80911E0229
:1016F00090911F02A0912002B09121020097A105B4
:10170000B10509F0FEC08091EB009091EC00A09132
:10171000ED00B091EE0024E630E040E050E0BC0186
:10172000CD010E94FC3CDA01C9019C01AD01809110
:10173000EE019091EF01A091F001B091F1018217BB
:101740009307A407B50708F0DCC08091EB009091E7
:10175000EC00A091ED00B091EE0024E630E040E016
:1017600050E0BC01CD010E94FC3CDA01C9019C01A2
:10177000AD018091EE019091EF01A091F001B09147
:10178000F10179018A01E81AF90A0A0B1B0BD80149
:10179000C701AC01BD0120917000309171008091B2
:1017A0006E0090916F00820F931FAA27BB278417AA
:1017B0009507A607B7070CF0A4C0209150033091FD
:1017C000510380916400909165008217930708F09F
:1017D00098C080919701909198019C0180919B0005
:1017E00090919C002817390708F08BC01A828091CD
:1017F0008B0190918C019C01809164009091650017
:1018000086509F4F8217930740F480916E0090910D
:101810006F00969587958A8319C080918B0190916E
:101820008C019C0180916400909165008A569F4FC5
:101830008217930758F480916E0090916F0025E015
:1018400030E0B9010E94D53CCB018A838A81282FE0
:10185000332727FD309580916E0090916F00820FA5
:10186000931FAC0160E070E081E00E94B91D80919F
:101870008B0190918C019093DF018093DE01809128
:10188000DA018F5F8093DA018091EA019091EB0198
:10189000A091EC01B091ED010196A11DB11D8093C5
:1018A000EA019093EB01A093EC01B093ED018091DC
:1018B000EB009091EC00A091ED00B091EE0024E6D9
:1018C00030E040E050E0BC01CD010E94FC3CDA0178
:1018D000C9018093EE019093EF01A093F001B093C2
:1018E000F10148E552E060E070E082E00E94B91D3D
:1018F0008091E901813029F48EE18093D501109225
:10190000E901209187013091880180917800992721
:101910002817390724F081E08093E90102C0109272
:10192000E90180918B0190918C01843691050CF036
:10193000CCC61092D501C9C61092760110927701DB
:10194000109278011092790180918B0190918C0115
:101950009C018091E0019091E1018217930740F48E
:1019600080918B0190918C019093E1018093E00133
:101970001092E20180917A008093E30180917A00D5
:101980008093E4018091E0019091E10102E08732CF
:10199000900740F080918B0190918C0182339105EA
:1019A0000CF434C180912A0290912B02A0912C0258
:1019B000B0912D022091EB003091EC004091ED00B0
:1019C0005091EE0028513C4F4F4F5F4F82179307C5
:1019D000A407B50738F440EB54E060E070E084E021
:1019E0000E94B91D80911A0290911B02A0911C02C5
:1019F000B0911D020097A105B10569F480918200A4
:101A0000909183002091840030918500AC01B90150
:101A100080E00E94B91D80911E0290911F02A0914A
:101A20002002B09121020097A105B10509F0EEC096
:101A30008091EB009091EC00A091ED00B091EE0050
:101A400024E630E040E050E0BC01CD010E94FC3CC7
:101A5000DA01C9019C01AD018091EE019091EF0185
:101A6000A091F001B091F10182179307A407B50787
:101A700008F0CCC08091EB009091EC00A091ED00BB
:101A8000B091EE0024E630E040E050E0BC01CD0132
:101A90000E94FC3CDA01C9019C01AD018091EE017C
:101AA0009091EF01A091F001B091F10179018A01CB
:101AB000E81AF90A0A0B1B0BD801C701AC01BD01DA
:101AC00020917E0030917F0080917C0090917D007C
:101AD000820F931FAA27BB2784179507A607B7076E
:101AE0000CF094C0209150033091510380918000FC
:101AF000909181008217930708F088C08091970128
:101B0000909198019C0180919B0090919C002817D6
:101B1000390708F07BC0198280918B0190918C016C
:101B20009C01809164009091650086509F4F8217C0
:101B3000930740F480917C0090917D009695879565
:101B4000898319C080918B0190918C019C018091B7
:101B50006400909165008A569F4F8217930758F44E
:101B600080917C0090917D0025E030E0B9010E94D9
:101B7000D53CCB0189838981282F332780917C0034
:101B800090917D00820F931FAC0160E070E081E0D6
:101B90000E94B91D48E552E060E070E082E00E94DA
:101BA000B91D80918B0190918C019093DF018093FE
:101BB000DE018091EA019091EB01A091EC01B091DE
:101BC000ED010196A11DB11D8093EA019093EB01F7
:101BD000A093EC01B093ED018091EB009091EC00AB
:101BE000A091ED00B091EE0024E630E040E050E03E
:101BF000BC01CD010E94FC3CDA01C9018093EE01D9
:101C00009093EF01A093F001B093F101409187010F
:101C10005091880180917800282F33278091790096
:101C200099278901081B190BC801481759072CF57A
:101C300080918B0190918C01803991051CF4109258
:101C4000D5011BC01092EA011092EB011092EC0139
:101C50001092ED011092D8011092D70180E280938A
:101C6000D5011092DF011092DE0180917700809300
:101C7000E301809177008093E40120918701309106
:101C800088018091780099270A96821793070CF0B3
:101C90001CC588E28093D50118C580917A00809395
:101CA000E30180917A008093E40120912202309137
:101CB000230240912402509125028091EB009091E3
:101CC000EC00A091ED00B091EE0088519C4FAF4F19
:101CD000BF4F281739074A075B0738F448E552E039
:101CE00060E070E082E00E94B91D80912A0290912C
:101CF0002B02A0912C02B0912D022091EB0030918B
:101D0000EC004091ED005091EE0028513C4F4F4FB8
:101D10005F4F82179307A407B50738F440EB54E0F0
:101D200060E070E084E00E94B91D8091EB0090912A
:101D3000EC00A091ED00B091EE0024E630E040E030
:101D400050E0BC01CD010E94FC3CDA01C9019C01BC
:101D5000AD018091D1019091D201A091D301B091B8
:101D6000D40182179307A407B50708F0AEC41092F8
:101D7000D5011092E201A9C480912A0290912B0210
:101D8000A0912C02B0912D022091EB003091EC003B
:101D90004091ED005091EE0028513C4F4F4F5F4F66
:101DA00082179307A407B50738F440EB54E060E0CE
:101DB00070E084E00E94B91D8091EA019091EB01EE
:101DC000A091EC01B091ED010097A105B10509F0DA
:101DD0005CC080911E0290911F02A0912002B091E0
:101DE00021020097A105B10509F04FC0809166005E
:101DF00090916700AC0160E070E083E00E94B91D43
:101E000048E552E060E070E082E00E94B91D8091F8
:101E10006E0090916F0025E030E0B9010E94D53C42
:101E2000CB01AC0160E070E081E00E94B91D8091BF
:101E3000EA019091EB01A091EC01B091ED010196C6
:101E4000A11DB11D8093EA019093EB01A093EC01D9
:101E5000B093ED018091EB009091EC00A091ED002A
:101E6000B091EE0024E630E040E050E0BC01CD014E
:101E70000E94FC3CDA01C9018093EE019093EF01CE
:101E8000A093F001B093F10127C08091EA019091F5
:101E9000EB01A091EC01B091ED0181309105A1051C
:101EA000B105D1F480911E0290911F02A0912002F1
:101EB000B09121020097A105B10571F48091DE0176
:101EC0009091DF01009741F480918B0190918C01FA
:101ED0009093DF018093DE0180918B0190918C01C2
:101EE0009C018091DE019091DF018C599F4F8217F8
:101EF000930708F01FC18091DE019091DF010097E8
:101F000009F418C184E690E09093DF018093DE012C
:101F1000809176008093E301809176008093E401C4
:101F20008091EA019091EB01A091EC01B091ED015B
:101F30000097A105B10509F4FDC08091EA019091D7
:101F4000EB01A091EC01B091ED018A309105A10562
:101F5000B10508F0EFC080911E0290911F02A09180
:101F60002002B09121020097A105B10509F0E2C05D
:101F700080918B0190918C018C018091EA0190916C
:101F8000EB01A091EC01B091ED0129E130E040E0DE
:101F900050E0BC01CD010E94B63CDC01CB019C01AC
:101FA0008091740090917500820F931F499780175C
:101FB000910708F0BFC08091EB009091EC00A091D8
:101FC000ED00B091EE0024E630E040E050E0BC01CE
:101FD000CD010E94FC3CDA01C9019C01AD01809158
:101FE000EE019091EF01A091F001B091F101790122
:101FF0008A01E81AF90A0A0B1B0BD801C7018333BF
:102000009105A105B10508F495C08091EB00909170
:10201000EC00A091ED00B091EE0024E630E040E04D
:1020200050E0BC01CD010E94FC3CDA01C9019C01D9
:10203000AD018091EE019091EF01A091F001B0917E
:10204000F10182179307A407B50708F073C08091C8
:102050009701909198019C0180919B0090919C0028
:102060002817390708F066C040E157E260E070E0E9
:1020700084E00E94B91D48E552E060E070E082E033
:102080000E94B91D80916A0090916B0020918D0093
:1020900030918E00AC01B90181E00E94B91D8091A0
:1020A000EA019091EB01A091EC01B091ED01019654
:1020B000A11DB11D8093EA019093EB01A093EC0167
:1020C000B093ED018091EB009091EC00A091ED00B8
:1020D000B091EE0024E630E040E050E0BC01CD01DC
:1020E0000E94FC3CDA01C9019C01AD0180918D0088
:1020F00090918E00AA27BB27280F391F4A1F5B1F0C
:1021000080916A0090916B00AA27BB27820F931FD2
:10211000A41FB51F8093EE019093EF01A093F001EF
:10212000B093F101809186009091870090938E008A
:1021300080938D008091EA019091EB01A091EC01D8
:10214000B091ED0187309105A105B105B8F18091FD
:102150001E0290911F02A0912002B09121020097CF
:10216000A105B10559F580918B0190918C019C01DD
:102170008091890090918A0082179307F8F4109259
:10218000EA011092EB011092EC011092ED018AE04D
:102190008093D5018091EE019091EF01A091F00123
:1021A000B091F10180559040A040B0408093EE0185
:1021B0009093EF01A093F001B093F10180918B0116
:1021C00090918C01803591050CF07FC21092D50161
:1021D0007CC21092760110927701109278011092D1
:1021E000790180917B008093E30180917B00809353
:1021F000E40180911E0290911F02A0912002B091F3
:1022000021020097A105B10539F040E050E060E0FF
:1022100070E081E00E94B91D80918B0190918C014A
:10222000893C91050CF47BC080912A0290912B028D
:10223000A0912C02B0912D022091EB003091EC0086
:102240004091ED005091EE0028513C4F4F4F5F4FB1
:1022500082179307A407B50738F440EB54E060E019
:1022600070E084E00E94B91D80911A0290911B02D7
:10227000A0911C02B0911D020097A105B10599F42F
:10228000409182005091830020918400309185001C
:10229000C901880F991F820F931F96958795BC01DE
:1022A00080E00E94B91D4091870150918801809182
:1022B0007800282F33278091790099278901081BFE
:1022C000190BC801481759070CF0FFC180918B0109
:1022D00090918C0111E0803991070CF0F6C11092B9
:1022E000EA011092EB011092EC011092ED011092B4
:1022F000EE011092EF011092F0011092F10180E2D4
:102300008093D5011092DF011092DE018091770059
:102310008093E301809177008093E401D6C14091DE
:1023200087015091880180917800282F3327809170
:1023300079009927B901681B790BCB014817590718
:102340000CF0C3C11092D5011092E201BEC1809180
:1023500076008093E401809176008093E301809180
:102360001A0290911B02A0911C02B0911D020097CD
:10237000A105B10569F480918200909183002091BC
:10238000840030918500AC01B90180E00E94B91D44
:1023900080912A0290912B02A0912C02B0912D02E3
:1023A0002091EB003091EC004091ED005091EE0057
:1023B00028513C4F4F4F5F4F82179307A407B50733
:1023C00038F440EB54E060E070E084E00E94B91D16
:1023D00080918B0190918C019C018091E001909102
:1023E000E1018217930740F480918B0190918C0159
:1023F0009093E1018093E00180918B0190918C0199
:102400009C018091E0019091E1018659904028174C
:10241000390740F080918B0190918C0172E08F3EE2
:1024200097072CF01092DA018DE38093D50180910B
:102430008B0190918C01843691050CF046C110926D
:10244000D50143C180911A0290911B02A0911C02F8
:10245000B0911D020097A105B10569F48091820039
:10246000909183002091840030918500AC01B901E6
:1024700080E00E94B91D80912A0290912B02A091C8
:102480002C02B0912D022091EB003091EC00409194
:10249000ED005091EE0028513C4F4F4F5F4F821797
:1024A0009307A407B50738F440EB54E060E070E010
:1024B00084E00E94B91D80911E0290911F02A0919C
:1024C0002002B09121020097A105B10509F0AAC030
:1024D0008091EB009091EC00A091ED00B091EE00A6
:1024E00024E630E040E050E0BC01CD010E94FC3C1D
:1024F000DA01C9019C01AD018091EE019091EF01DB
:10250000A091F001B091F10182179307A407B507DC
:1025100008F088C08091EB009091EC00A091ED0054
:10252000B091EE0024E630E040E050E0BC01CD0187
:102530000E94FC3CDA01C9019C01AD018091EE01D1
:102540009091EF01A091F001B091F101BA01A901C0
:10255000481B590B6A0B7B0B8091700090917100A6
:102560009C01220F331F80916E0090916F00820FAB
:10257000931FAA27BB2784179507A607B70708F05C
:1025800051C080918B0190918C019C0180916400DD
:10259000909165008217930708F044C080916E0007
:1025A00090916F00AC0160E070E081E00E94B91D85
:1025B00080918B0190918C019093DF018093DE01DB
:1025C0008091DA018F5F8093DA018091EA01909126
:1025D000EB01A091EC01B091ED010196A11DB11D9F
:1025E0008093EA019093EB01A093EC01B093ED018D
:1025F0008091EB009091EC00A091ED00B091EE0085
:1026000024E630E040E050E0BC01CD010E94FC3CFB
:10261000DA01C9018093EE019093EF01A093F001DC
:10262000B093F1018091DA01843028F01092DA0140
:1026300083E18093D50120918701309188018091B9
:1026400078009927821793071CF48EE18093D501B7
:1026500080918B0190918C0184369105B4F5109294
:10266000D50133C01092E3011092E40180911E0263
:1026700090911F02A0912002B09121020097A10524
:10268000B10539F040E050E060E070E081E00E9488
:10269000B91D80912A0290912B02A0912C02B09139
:1026A0002D020097A105B10539F041E050E060E04E
:1026B00070E084E00E94B91D82E090E09093E80110
:1026C0008093E70102C01092D50180914C028833BB
:1026D00098F010924C0280E592E00E941E2D80ED51
:1026E00092E00E941E2D8091420290914302019639
:1026F0009093430280934202A89580917C0181309F
:1027000009F0A2C310927C0180917B01843009F012
:10271000B9C08091AB019091AC01A091AD01B09195
:10272000AE0126E636E646E65FE3BC01CD010E9437
:102730006E3CDC01CB018FA398A7A9A7BAA7E4E25E
:10274000F0E000811181C801AA2797FDA095BA2F5A
:10275000BC01CD010E94F43B6BA37CA38DA39EA37F
:10276000112384F420E030E040E857E46BA17CA121
:102770008DA19EA10E944F3BDC01CB018BA39CA3AA
:10278000ADA3BEA320E932EC45EF5DE36BA17CA1D4
:102790008DA19EA10E946E3CDC01CB019C01AD018C
:1027A0006FA178A589A59AA50E944F3BDC01CB01BA
:1027B0008093AB019093AC01A093AD01B093AE01B7
:1027C0008091AB019091AC01A091AD01B091AE01AF
:1027D000BC01CD010E94D73BDC01CB0190938C0161
:1027E00080938B0180918B0190918C019093510388
:1027F00080935003209152033091530380915003F2
:1028000090915103820F931F969587959093530350
:1028100080935203209154033091550380915203C9
:1028200090915303820F931F96958795909355032C
:102830008093540381E080937B0180918B01909180
:102840008C01AA2797FDA095BA2FBC01CD010E944B
:10285000F43BDC01CB018093080390930903A09320
:102860000A03B0930B03EBE3F0E080818F7D80835C
:10287000EBE3F0E080818F7E8083E7E2F0E081E0AF
:102880008083E2C280917B01813039F486E08093BD
:102890007B01E7E2F0E01082D7C280917B018530B6
:1028A00009F07BC08091AF019091B001A091B1017E
:1028B000B091B2012DEC3CEC4CE45FE3BC01CD01E6
:1028C0000E946E3CDC01CB018F8F98A3A9A3BAA311
:1028D000E4E2F0E000811181C801AA2797FDA095EC
:1028E000BA2FBC01CD010E94F43B6B8F7C8F8D8F82
:1028F0009E8F112384F420E030E040E857E46B8D94
:102900007C8D8D8D9E8D0E944F3BDC01CB018B8F8A
:102910009C8FAD8FBE8F20E932EC45E75EE36B8D77
:102920007C8D8D8D9E8D0E946E3CDC01CB019C01C7
:10293000AD016F8D78A189A19AA10E944F3BDC0166
:10294000CB018093AF019093B001A093B101B093FC
:10295000B2018091AF019091B001A091B101B0910D
:10296000B201BC01CD010E94D73BDC01CB019093A9
:102970008E0180938D0182E080937B01EBE3F0E098
:10298000808180628083EBE3F0E0808180618083DE
:10299000E7E2F0E082E0808357C280917B018230E1
:1029A00069F580919701909198019093900180939F
:1029B0008F012091970130919801C901880F991FCB
:1029C000880F991F880F991F821B930B9C01E4E2CB
:1029D000F0E080819181820F931F9695879596955F
:1029E000879596958795909398018093970187E0B6
:1029F00080937B01E7E2F0E0108226C280917B01A8
:102A0000863089F410927B01EBE3F0E080818062F4
:102A10008083EBE3F0E080818F7E8083E7E2F0E06B
:102A200083E0808311C280917B01882309F0C6C0B6
:102A300080919B0190919C01A0919D01B0919E017C
:102A400023E333E343E75FE3BC01CD010E946E3C27
:102A5000DC01CB018F8B988FA98FBA8FE4E2F0E075
:102A600000811181C801AA2797FDA095BA2FBC014A
:102A7000CD010E94F43B6B8B7C8B8D8B9E8B112345
:102A800084F420E030E040E857E46B897C898D894C
:102A90009E890E944F3BDC01CB018B8B9C8BAD8BC5
:102AA000BE8B2DEC3CEC4CE45DE36B897C898D891D
:102AB0009E890E946E3CDC01CB019C01AD016F89B7
:102AC000788D898D9A8D0E944F3BDC01CB018093DC
:102AD0009B0190939C01A0939D01B0939E018091D6
:102AE0009B0190919C01A0919D01B0919E01BC0120
:102AF000CD010E94D73BDC01CB01909384018093F0
:102B0000830185E080937B01809183019091840112
:102B1000AA2797FDA095BA2FBC01CD010E94F43BD6
:102B20007B018C018091930090919400A09195007D
:102B3000B09196009C01AD01C801B7010E946E3CA6
:102B4000DC01CB018093CB019093CC01A093CD010C
:102B5000B093CE01E090CB01F090CC010091CD017B
:102B60001091CE018091970090919800A0919900CA
:102B7000B0919A009C01AD01C801B7010E944E3B83
:102B8000DC01CB018093CB019093CC01A093CD01CC
:102B9000B093CE018091CB019091CC01A091CD0159
:102BA000B091CE018093880290938902A0938A020B
:102BB000B0938B02E7E2F0E0108246C180917B0186
:102BC000873009F03FC02091910130919201C901F5
:102BD000880F991F880F991F880F991F821B930BCD
:102BE0008C01E4E2F0E020813181C901880F991F56
:102BF000820F931F880F991F880F991F2AE030E0DA
:102C0000B9010E94D53CCB01800F911F9695879505
:102C100096958795969587959093920180939101CB
:102C200083E080937B01EBE3F0E080818F7D808304
:102C3000EBE3F0E0808180618083E7E2F0E086E012
:102C4000808302C180917B01833009F079C080913B
:102C5000A7019091A801A091A901B091AA012DEC22
:102C60003CEC4CE45FE3BC01CD010E946E3CDC0116
:102C7000CB018F87988BA98BBA8BE4E2F0E00081BF
:102C80001181C801AA2797FDA095BA2FBC01CD01DB
:102C90000E94F43B6B877C878D879E87112384F489
:102CA00020E030E040E857E46B857C858D859E858B
:102CB0000E944F3BDC01CB018B879C87AD87BE8791
:102CC0002DEC3CEC4CE45EE36B857C858D859E852C
:102CD0000E946E3CDC01CB019C01AD016F857889BF
:102CE00089899A890E944F3BDC01CB018093A7011F
:102CF0009093A801A093A901B093AA018091A70184
:102D00009091A801A091A901B091AA01BC01CD01A7
:102D10000E94D73BDC01CB0190938A01809389010B
:102D200088E080937B0183E00E944E209927909356
:102D3000880180938701E7E2F0E087E0808384C028
:102D400080917B01883009F078C08091BB0190911F
:102D5000BC01A091BD01B091BE012DEC3CEC4CE456
:102D60005FE3BC01CD010E946E3CDC01CB018F838F
:102D70009887A987BA87E4E2F0E000811181C80151
:102D8000AA2797FDA095BA2FBC01CD010E94F43B64
:102D90006B837C838D839E83112384F420E030E059
:102DA00040E857E46B817C818D819E810E944F3B7E
:102DB000DC01CB018B839C83AD83BE832DEC3CEC8B
:102DC0004CE45EE36B817C818D819E810E946E3C30
:102DD000DC01CB019C01AD016F81788589859A85E5
:102DE0000E944F3BDC01CB018093BB019093BC015F
:102DF000A093BD01B093BE018091BB019091BC0135
:102E0000A091BD01B091BE01BC01CD010E94D73B94
:102E1000DC01CB01909394018093930184E0809333
:102E20007B0188E00E944E20992790938601809331
:102E30008501E7E2F0E0108207C010927B01E7E233
:102E4000F0E080917B0180830E94821E0E9410200E
:102E50000C940002CF93DF93CDB7DEB7C257D040BA
:102E60000FB6F894DEBF0FBECDBFFE01E059FF4F95
:102E700085E090E091838083FE01E059FF4FA081BF
:102E8000B1810E941E3D802DFE01E059FF4FB183AC
:102E9000A083FE01EE58FF4F8083FE01EE58FF4FE6
:102EA000808199278F3F09F443C4FE01E359FF4F06
:102EB00084E090E091838083FE01E359FF4FA0817D
:102EC000B1810E941E3D802DFE01E359FF4FB18369
:102ED000A083FE01E159FF4F8083FE01E159FF4FBE
:102EE00080819927282F3327FE01E659FF4F85E07F
:102EF00090E091838083FE01E659FF4FA081B1816C
:102F00000E941E3D802DFE01E659FF4FB183A08334
:102F1000FE01E459FF4F8083FE01E459FF4F808199
:102F200099279927982F8827820F931F90936500E0
:102F300080936400FE01E959FF4F86E090E09183A1
:102F40008083FE01E959FF4FA081B1810E941E3D9F
:102F5000802DFE01E959FF4FB183A083FE01E7599F
:102F6000FF4F8083FE01E759FF4F80819927282F6B
:102F70003327FE01EC59FF4F87E090E09183808377
:102F8000FE01EC59FF4FA081B1810E941E3D802DB2
:102F9000FE01EC59FF4FB183A083FE01EA59FF4FB8
:102FA0008083FE01EA59FF4F808199279927982F46
:102FB0008827820F931F9C01220F331FC901880F9E
:102FC000991F880F991F820F931F909383008093FE
:102FD0008200FE01EF59FF4F88E090E091838083EB
:102FE000FE01EF59FF4FA081B1810E941E3D802D4F
:102FF000FE01EF59FF4FB183A083FE01ED59FF4F52
:103000008083FE01ED59FF4F80819927282F3327B8
:10301000FE01E25AFF4F89E090E091838083FE0138
:10302000E25AFF4FA081B1810E941E3D802DFE011A
:10303000E25AFF4FB183A083FE01E05AFF4F808325
:10304000FE01E05AFF4F808199279927982F882702
:10305000820F931F9C01220F331FC901880F991FF4
:10306000880F991F820F931F9093670080936600CB
:10307000FE01E55AFF4F8AE090E091838083FE01D4
:10308000E55AFF4FA081B1810E941E3D802DFE01B7
:10309000E55AFF4FB183A083FE01E35AFF4F8083BF
:1030A000FE01E35AFF4F80819927282F3327FE0125
:1030B000E85AFF4F8BE090E091838083FE01E85A4D
:1030C000FF4FA081B1810E941E3D802DFE01E85A74
:1030D000FF4FB183A083FE01E65AFF4F8083FE01BC
:1030E000E65AFF4F808199279927982F8827820FCA
:1030F000931F9C01220F331FC901880F991F880F4E
:10310000991F820F931F9093690080936800FE01BE
:10311000EB5AFF4F8CE090E091838083FE01EB5AE5
:10312000FF4FA081B1810E941E3D802DFE01EB5A10
:10313000FF4FB183A083FE01E95AFF4F8083FE0158
:10314000E95AFF4F80819927282F3327FE01EE5A35
:10315000FF4F8DE090E091838083FE01EE5AFF4F98
:10316000A081B1810E941E3D802DFE01EE5AFF4FCD
:10317000B183A083FE01EC5AFF4F8083FE01EC5A1D
:10318000FF4F808199279927982F8827820F931FB7
:103190009C01220F331FC901880F991F880F991FA7
:1031A000820F931F90936B0080936A00FE01E15B96
:1031B000FF4F8EE090E091838083FE01E15BFF4F43
:1031C000A081B1810E941E3D802DFE01E15BFF4F79
:1031D000B183A083FE01EF5AFF4F8083FE01EF5AB7
:1031E000FF4F80819927282F3327FE01E45BFF4F93
:1031F0008FE090E091838083FE01E45BFF4FA0812C
:10320000B1810E941E3D802DFE01E45BFF4FB18322
:10321000A083FE01E25BFF4F8083FE01E25BFF4F74
:10322000808199279927982F8827820F931F9C01C7
:10323000220F331FC901880F991F880F991F820F12
:10324000931F90936F0080936E00FE01E75BFF4F2A
:1032500080E190E091838083FE01E75BFF4FA081D6
:10326000B1810E941E3D802DFE01E75BFF4FB183BF
:10327000A083FE01E55BFF4F8083FE01E55BFF4F0E
:1032800080819927282F3327FE01EA5BFF4F81E1D8
:1032900090E091838083FE01EA5BFF4FA081B181C2
:1032A0000E941E3D802DFE01EA5BFF4FB183A0838B
:1032B000FE01E85BFF4F8083FE01E85BFF4F8081EA
:1032C00099279927982F8827820F931F90939C0006
:1032D00080939B00FE01ED5BFF4F82E190E09183C4
:1032E0008083FE01ED5BFF4FA081B1810E941E3DF6
:1032F000802DFE01ED5BFF4FB183A083FE01EB5BF0
:10330000FF4F8083FE01EB5BFF4F80819927282FC1
:103310003327FE01E05CFF4F83E190E091838083DF
:10332000FE01E05CFF4FA081B1810E941E3D802D17
:10333000FE01E05CFF4FB183A083FE01EE5BFF4F17
:103340008083FE01EE5BFF4F808199279927982F9C
:103350008827820F931F9C01220F331FC901880FFA
:10336000991F880F991F820F931F9093710080936C
:10337000700084EB90E0909375008093740084E17A
:1033800090E09EAF8DAFADADBEAD0E941E3D802DD5
:10339000BEAFADAF8FAF8FAD9927282F332785E113
:1033A00090E09BAF8AAFAAADBBAD0E941E3D802DC1
:1033B000BBAFAAAF8CAF8CAD99279927982F8827E0
:1033C000820F931F9C01220F331FC901880F991F81
:1033D000880F991F820F931F90938500809384001C
:1033E00086E190E098AF8FABAFA9B8AD0E941E3DCB
:1033F000802DB8AFAFAB89AF89AD9927282F332780
:1034000087E190E09DAB8CABACA9BDA90E941E3DAD
:10341000802DBDABACAB8EAB8EA999279927982F89
:103420008827820F931F909373008093720088E126
:1034300090E09AAB89ABA9A9BAA90E941E3D802D44
:10344000BAABA9AB8BAB8BA999278093760089E1A6
:1034500090E09FA78EA7AEA5BFA50E941E3D802D20
:10346000BFA7AEA788AB88A99927809377008AE188
:1034700090E09CA78BA7ABA5BCA50E941E3D802D0C
:10348000BCA7ABA78DA78DA59927809378008BE16A
:1034900090E099A788A7A8A5B9A50E941E3D802DF8
:1034A000B9A7A8A78AA78AA59927809379008CE154
:1034B00090E09EA38DA3ADA1BEA10E941E3D802DD4
:1034C000BEA3ADA38FA38FA1992780937A008DE12E
:1034D00090E09BA38AA3AAA1BBA10E941E3D802DC0
:1034E000BBA3AAA38CA38CA1992780937B008EE118
:1034F00090E098A38F8FAF8DB8A10E941E3D802DC4
:10350000B8A3AF8F89A389A19927282F33278FE1EB
:1035100090E09D8F8C8FAC8DBD8D0E941E3D802DC7
:10352000BD8FAC8F8E8F8E8D99279927982F8827E6
:10353000820F931F9C01220F331FC901880F991F0F
:10354000880F991F820F931F90937D0080937C00BA
:1035500080E290E09A8F898FA98DBA8D0E941E3DDE
:10356000802DBA8FA98F8B8F8B8D9927282F33278A
:1035700081E290E09F8B8E8BAE89BF890E941E3DB9
:10358000802DBF8BAE8B888F888D99279927982F98
:103590008827820F931F9C01220F331FC901880FB8
:1035A000991F880F991F820F931F90937F0080931C
:1035B0007E0082E290E09C8B8B8BAB89BC890E9461
:1035C0001E3D802DBC8BAB8B8D8B8D899927282F31
:1035D000332783E290E0998B888BA889B9890E9470
:1035E0001E3D802DB98BA88B8A8B8A8999279927B4
:1035F000982F8827820F931F9093810080938000DB
:1036000084E290E09E878D87AD85BE850E941E3D39
:10361000802DBE87AD878F878F85992799279C013D
:10362000220F331FC901880F991F880F991F820F1E
:10363000931F909387008093860085E290E09B879C
:103640008A87AA85BB850E941E3D802DBB87AA87DD
:103650008C878C8599278093880086E290E09887F4
:103660008F83AF81B8850E941E3D802DB887AF83C0
:1036700089878985992799279C01220F331FC901C2
:10368000880F991F880F991F820F931F90938E00A8
:1036900080938D0087E290E09D838C83AC81BD8117
:1036A0000E941E3D802DBD83AC838E838E81992721
:1036B00099279C01220F331FC901880F991F880F7A
:1036C000991F820F931F90938A008093890088E24C
:1036D00090E09A838983A981BA810E941E3D802D42
:1036E000BA83A9838B838B81992799279C01220F09
:1036F000331FC901880F991F880F991F820F931FCD
:1037000090938C0080938B00209164003091650031
:103710008091720090917300A901481B590BCA0156
:1037200026E030E0B9010E94D53CCB0180938F00A8
:10373000EFE3F0E01082EEE3F0E01082CE58DF4FCE
:103740000FB6F894DEBF0FBECDBFDF91CF910895C5
:10375000CF93DF93CDB7DEB784E690E09093CF02AE
:103760008093CE0288EC90E090934F0380934E03B9
:1037700080E090E0A7EDB3E48093D8029093D90263
:10378000A093DA02B093DB0280ED92E00E94A928B8
:1037900080E090E0A0EAB0E4809358029093590250
:1037A000A0935A02B0935B0280E592E00E94A928A0
:1037B00010925402EFE3F0E01082EEE3F0E01082AA
:1037C000DF91CF910895CF93DF93CDB7DEB7DF912F
:1037D000CF910895EF92FF920F931F93CF93DF93B2
:1037E000CDB7DEB725970FB6F894DEBF0FBECDBFBD
:1037F0001A821B821C821D82F8948091EB009091AA
:10380000EC00A091ED00B091EE008A839B83AC8325
:10381000BD83789419821982B5C089819927880F50
:10382000991F880F991FFC01EE50FE4F80819181F6
:10383000A281B3810097A105B105D9F189819927AA
:10384000880F991F880F991FFC01EE50FE4F2081B1
:103850003181428153818A819B81AC81BD818217F4
:103860009307A407B50728F58981682F77278981F1
:103870009927880F991F880F991FFC01EE50FE4F62
:1038800020813181428153818A819B81AC81BD81BC
:10389000281B390B4A0B5B0BCB01880F991F880F34
:1038A000991FFC01EE50FE4F2083318342835383E6
:1038B0000DC089819927880F991F880F991FFC01D6
:1038C000EE50FE4F10821182128213828981992755
:1038D000880F991F880F991FFC01E65EFD4F8081BC
:1038E0009181A281B3810097A105B105D9F18981A8
:1038F0009927880F991F880F991FFC01E65EFD4FDD
:1039000020813181428153818A819B81AC81BD813B
:1039100082179307A407B50728F58981682F7727B1
:1039200089819927880F991F880F991FFC01E65EEE
:10393000FD4F20813181428153818A819B81AC81FD
:10394000BD81281B390B4A0B5B0BCB01880F991FDC
:10395000880F991FFC01E65EFD4F2083318342836F
:1039600053830DC089819927880F991F880F991F4C
:10397000FC01E65EFD4F1082118212821382898162
:103980008F5F898389818A3008F447CF10920202C1
:1039900010920302109204021092050210922A0261
:1039A00010922B0210922C0210922D0210920602FD
:1039B00010920702109208021092090210922E0231
:1039C00010922F02109230021092310210920A02CD
:1039D00010920B0210920C0210920D021092320201
:1039E00010923302109234021092350210920E029D
:1039F00010920F02109210021092110210923602D1
:103A0000109237021092380210923902109212026C
:103A100010921302109214021092150210923A02A0
:103A200010923B0210923C0210923D02109216023C
:103A300010921702109218021092190210923E0270
:103A400010923F02109240021092410220917601A2
:103A50003091770140917801509179018A819B8161
:103A6000AC81BD8179018A01E81AF90A0A0B1B0BA6
:103A7000D801C7018093760190937701A0937801D4
:103A8000B09379011092EE011092EF011092F001C3
:103A90001092F10184E690E0A0E0B0E08093D101C3
:103AA0009093D201A093D301B093D4018CE80E94EB
:103AB000F82585E00E94F82589E00E94F82580918C
:103AC000D50180680E94F8258A819B81AC81BD81E7
:103AD00024E630E040E050E0BC01CD010E94FC3C17
:103AE000DA01C9010E94F8258A819B81AC81BD81E0
:103AF00024E630E040E050E0BC01CD010E94FC3CF7
:103B0000DA01C901892F9A2FAB2FBB270E94F82514
:103B10008A819B81AC81BD8124E630E040E050E0A9
:103B2000BC01CD010E94FC3CDA01C901CD01AA27EC
:103B3000BB270E94F82583E70E94F825F89484E1CA
:103B400090E0A0E0B0E08093EB009093EC00A093B5
:103B5000ED00B093EE00789425960FB6F894DEBF92
:103B60000FBECDBFDF91CF911F910F91FF90EF90CE
:103B70000895CF93DF93CDB7DEB729970FB6F894AA
:103B8000DEBF0FBECDBF8D837F836E83598748878D
:103B9000F8948091DB01882361F08D81813049F4B4
:103BA0008091D501893029F088859985009709F0A1
:103BB0009FC019821A821B821C828E819F81AA2734
:103BC000BB2789839A83AB83BC8389819A81AB812C
:103BD000BC812AE030E040E050E0BC01CD010E9411
:103BE000B63CDC01CB0189839A83AB83BC8389819A
:103BF0009A81AB81BC812AE030E040E050E0BC011A
:103C0000CD010E94B63CDC01CB0189839A83AB8352
:103C1000BC838D81682F77272091EB003091EC00D9
:103C20004091ED005091EE0089819A81AB81BC8179
:103C3000280F391F4A1F5B1FCB01880F991F880F60
:103C4000991FFC01EE50FE4F208331834283538342
:103C500088859985AA27BB2789839A83AB83BC83F0
:103C600089819A81AB81BC812AE030E040E050E05C
:103C7000BC01CD010E94B63CDC01CB0189839A8353
:103C8000AB83BC8389819A81AB81BC812AE030E01F
:103C900040E050E0BC01CD010E94B63CDC01CB010C
:103CA00089839A83AB83BC838D81682F77278D812D
:103CB0009927880F991F880F991FFC01EE50FE4F1E
:103CC000208131814281538189819A81AB81BC817C
:103CD000280F391F4A1F5B1FCB01880F991F880FC0
:103CE000991FFC01E65EFD4F20833183428353839D
:103CF000789429960FB6F894DEBF0FBECDBFDF9142
:103D0000CF910895CF93DF93CDB7DEB721970FB64C
:103D1000F894DEBF0FBECDBFF8948091EB00909178
:103D2000EC00A091ED00B091EE00809344029093DE
:103D30004502A0934602B0934702789419821982F3
:103D400062C189819927880F991F880F991FFC01EB
:103D5000EE50FE4F80819181A281B3810097A10531
:103D6000B10509F49CC089819927880F991F880F94
:103D7000991FFC01EE50FE4F208131814281538119
:103D80008091440290914502A0914602B091470271
:103D9000281739074A075B0708F081C089819927EE
:103DA000880F991FFC01E151FF4FA081B1818981EA
:103DB0009927880F991FFC01E151FF4F0190F08175
:103DC000E02D208189819927FC01ED5FFE4F8081E4
:103DD000822B8C9389819927880F991F880F991FAF
:103DE000FC01EE50FE4F10821182128213828981F3
:103DF000883008F054C08CE80E94F82585E00E94C5
:103E0000F82589810E94F8258091D50180680E945B
:103E1000F8258091440290914502A0914602B0910C
:103E2000470224E630E040E050E0BC01CD010E94B2
:103E3000FC3CDA01C9010E94F8258091440290916E
:103E40004502A0914602B091470224E630E040E0EE
:103E500050E0BC01CD010E94FC3CDA01C901892F70
:103E60009A2FAB2FBB270E94F82580914402909196
:103E70004502A0914602B091470224E630E040E0BE
:103E800050E0BC01CD010E94FC3CDA01C901CD012A
:103E9000AA27BB270E94F82583E70E94F82589817D
:103EA0009927880F991F880F991FFC01E65EFD4F27
:103EB00080819181A281B3810097A105B10509F4A8
:103EC0009FC089819927880F991F880F991FFC012E
:103ED000E65EFD4F20813181428153818091440211
:103EE00090914502A0914602B091470228173907E8
:103EF0004A075B0708F084C089819927880F991FBA
:103F0000FC01E151FF4FA081B18189819927880F80
:103F1000991FFC01E151FF4F0190F081E02D80815C
:103F2000282F89819927FC01ED5FFE4F80818095C4
:103F300082238C938981883008F055C08CE80E94D8
:103F4000F82585E00E94F82589810E94F825909146
:103F5000D5018FE789230E94F82580914402909132
:103F60004502A0914602B091470224E630E040E0CD
:103F700050E0BC01CD010E94FC3CDA01C9010E9465
:103F8000F8258091440290914502A0914602B0919B
:103F9000470224E630E040E050E0BC01CD010E9441
:103FA000FC3CDA01C901892F9A2FAB2FBB270E9455
:103FB000F8258091440290914502A0914602B0916B
:103FC000470224E630E040E050E0BC01CD010E9411
:103FD000FC3CDA01C901CD01AA27BB270E94F825C4
:103FE00083E70E94F82589819927880F991F880FF8
:103FF000991FFC01E65EFD4F10821182128213822E
:1040000089818F5F898389818A3008F49ACE2196CD
:104010000FB6F894DEBF0FBECDBFDF91CF910895EC
:104020000F931F93CF93DF93CDB7DEB721970FB6D2
:10403000F894DEBF0FBECDBF19820E947D26898312
:104040001092D60189818823E1F00FC08091D601BA
:10405000082F11270E94B025F801E95AFC4F8083F0
:104060008091D6018F5F8093D6019091D60189818E
:10407000981760F32091D60187E593E0622F0E94A4
:1040800072361092D60121960FB6F894DEBF0FBE9D
:10409000CDBFDF91CF911F910F910895CF93DF9303
:1040A000CDB7DEB728970FB6F894DEBF0FBECDBFF1
:1040B0008E831D828E819927880F991FFC01ED57F1
:1040C000FE4F8081918123E0833F92071CF0188688
:1040D0001F8287C08E819927880F991FFC01ED5799
:1040E000FE4F8081918133E08F3D93070CF471C0C6
:1040F00088ED90E098878F8374C08E819927880F10
:10410000991FFC01ED57FE4F808191819C018D81AB
:104110009927880F991FFC01E356FF4F80819181F9
:104120008217930708F052C01C821B828D81282FB2
:104130003327C901880F991F880F991F820F931F7A
:104140008D979C838B831A8219828D819927019781
:10415000880F991FFC01E356FF4F208131818E812A
:104160009927880F991FFC01ED57FE4F808191819F
:10417000281B390BC901880F991F880F991FAC01A3
:10418000420F531F8D8199270197880F991FFC01BA
:10419000E356FF4F208131818D819927880F991F28
:1041A000FC01E356FF4F80819181281B390BCA0126
:1041B000B9010E94D53CCB019A8389839B81898177
:1041C000890F282F332738872F830BC08D818F5F6E
:1041D0008D838D81873208F490CF86E990E09887AF
:1041E0008F838F81988528960FB6F894DEBF0FBE17
:1041F000CDBFDF91CF910895CF93DF93CDB7DEB7D9
:1042000088E10FB6F89481BD11BC0FBE0E94D5376E
:104210008DE091E00E947E3884E60E94B92780916B
:1042200083019091840183539140AA2797FDA09523
:10423000BA2FBC01CD010E94F43BDC01CB019C01F3
:10424000AD0163E373E387EA91E40E94913BDC01F3
:10425000CB018093930090939400A0939500B0932A
:1042600096008091930090919400A0919500B09158
:10427000960020E030E849E953E4BC01CD010E94FA
:104280006E3CDC01CB018093970090939800A09343
:104290009900B0939A0083E990E06CE271E00E948B
:1042A000222887E990E060E371E00E94222888E1FB
:1042B00090E02DE00FB6F894A89581BD0FBE21BD0A
:1042C00084E60E94B927DF91CF910895CF93DF93C1
:1042D000CDB7DEB78091CF019091D0010196909338
:1042E000D0018093CF018091CF019091D0010097B0
:1042F00011F40E94903780914802909149028230D7
:1043000091050CF451C00E94D5378AE191E00E94DA
:104310007E388091CB019091CC01A091CD01B091DC
:10432000CE0120E030E048EC52E4BC01CD010E9417
:104330006E3CDC01CB01BC01CD010E94D73BDC010E
:10434000CB0190934902809348028091480290915A
:10435000490246E062E00E947D3A8EE191E00E94CF
:104360007E388091D501992742E060E00E94DD39D6
:1043700084E291E00E947E3880918B0190918C01C3
:1043800044E060E00E94DD3988E291E00E947E38DE
:1043900080918D0190918E0144E060E00E94DD39B2
:1043A000109249021092480280914802909149026D
:1043B00001969093490280934802DF91CF9108952E
:1043C000CF93DF93CDB7DEB722970FB6F894DEBF59
:1043D0000FBECDBF80913A0290913B02A0913C026A
:1043E000B0913D020097A105B10509F075C080911B
:1043F000D501282F33273A83298389819A818E31E9
:10440000910509F442C029813A812F31310584F4A4
:1044100089819A818A30910541F129813A8124313B
:10442000310559F189819A8189309105B1F054C0E3
:1044300029813A8120323105C1F189819A81803206
:1044400091055CF129813A8128323105B1F18981E8
:104450009A8183369105C9F13FC04AE050E06AE095
:1044600070E088E00E94B91D37C045E050E065E08B
:1044700070E088E00E94B91D2FC042E350E060E088
:1044800070E088E00E94B91D27C04AE050E06EE16C
:1044900070E088E00E94B91D1FC04AE050E064E16E
:1044A00070E088E00E94B91D17C04AE050E064E166
:1044B00070E088E00E94B91D0FC04AE050E062E35E
:1044C00070E088E00E94B91D07C04AE050E064E651
:1044D00070E088E00E94B91D80913E0290913F02F9
:1044E000A0914002B09141020097A105B105D1F51C
:1044F0008091E7019091E801009741F440E050E09D
:1045000060E070E089E00E94B91D1DC08091E70164
:104510009091E8018130910541F44AE050E064E176
:1045200070E089E00E94B91D0EC08091E701909172
:10453000E8018230910539F44AE050E06AE070E029
:1045400089E00E94B91D80918B0190918C0124E03B
:104550008D3492073CF04AE050E060E070E089E082
:104560000E94B91D22960FB6F894DEBF0FBECDBFD4
:10457000DF91CF910895CF93DF93CDB7DEB7E3E519
:10458000F0E01082A9E5B0E0E9E5F0E08081836029
:104590008C93A3E5B0E0E3E5F0E0808183608C9349
:1045A000ECE5F0E01082A1E3B0E0E1E3F0E080812F
:1045B00080618C93A1E3B0E0E1E3F0E08081806270
:1045C0008C93E2E3F0E080818F7E8083E2E3F0E091
:1045D00080818F7D8083DF91CF9108951F920F920C
:1045E0000FB60F9211242F933F935F936F937F9396
:1045F0008F939F93AF93BF93EF93FF93CF93DF93EB
:10460000CDB7DEB72197DEBFCDBFF894E2E3F0E08F
:10461000808180618083E2E3F0E08081806280833A
:1046200080914B028F5F80934B0280914B028734C5
:10463000B0F110924B028091E401282F3327C90179
:10464000880F991F820F931F880F991F880F991F3A
:10465000880F991F820F931F2AE030E0B9010E9452
:10466000D53CCB018B5F8983ECE5F0E090818981BB
:10467000981740F4ACE5B0E0ECE5F0E080818F5FA6
:104680008C930DC0ECE5F0E090818981891738F4B6
:10469000ACE5B0E0ECE5F0E0808181508C9378945B
:1046A0002196F894DEBFCDBFDF91CF91FF91EF91BE
:1046B000BF91AF919F918F917F916F915F913F914A
:1046C0002F910F900FBE0F901F9018951F920F9271
:1046D0000FB60F9211248F939F93AF93BF93EF93D5
:1046E000FF93CF93DF93CDB7DEB7F89480912A0282
:1046F00090912B02A0912C02B0912D020097A10560
:10470000B10551F0E2E3F0E080818F7D8083E2E348
:10471000F0E080818F7E80837894DF91CF91FF914C
:10472000EF91BF91AF919F918F910F900FBE0F901E
:104730001F901895CF93DF93CDB7DEB7E5E4F0E097
:104740001082A9E5B0E0E9E5F0E0808180648C9317
:10475000A5E4B0E0E5E4F0E0808187608C93E4E4D8
:10476000F0E081E08083DF91CF9108951F920F9256
:104770000FB60F9211248F939F93AF93BF93CF9354
:10478000DF93CDB7DEB781E080937C018091EB00B1
:104790009091EC00A091ED00B091EE004296A11D29
:1047A000B11D8093EB009093EC00A093ED00B093CB
:1047B000EE0080914C028F5F80934C02DF91CF918D
:1047C000BF91AF919F918F910F900FBE0F901F904F
:1047D00018951F920F920FB60F9211248F939F93EB
:1047E000AF93BF93EF93FF93CF93DF93CDB7DEB734
:1047F00080914A02813069F410924A02AAE4B0E042
:10480000EAE4F0E0808191818C599F4F11969C934E
:104810008E93DF91CF91FF91EF91BF91AF919F91D7
:104820008F910F900FBE0F901F9018951F920F92AF
:104830000FB60F921124CF93DF93CDB7DEB7DF9180
:10484000CF910F900FBE0F901F9018951F920F924F
:104850000FB60F921124CF93DF93CDB7DEB7DF9160
:10486000CF910F900FBE0F901F9018951F920F922F
:104870000FB60F921124CF93DF93CDB7DEB7DF9140
:10488000CF910F900FBE0F901F9018951F920F920F
:104890000FB60F9211242F933F935F936F937F93E3
:1048A0008F939F93AF93BF93EF93FF93CF93DF9338
:1048B000CDB7DEB72297DEBFCDBFECE4F0E080815C
:1048C00091819A838983ECE4F0E0118210828091D7
:1048D0002D0190912E019C01220F331F220F331FB7
:1048E00089819A81820F931F880F991F2AE030E0F7
:1048F000B9010E94D53CCB0190932E0180932D01EC
:104900002296F894DEBFCDBFDF91CF91FF91EF915A
:10491000BF91AF919F918F917F916F915F913F91E7
:104920002F910F900FBE0F901F901895CF93DF938C
:10493000CDB7DEB7EFE4F0E01082EAE4F0E088E81B
:1049400093E191838083E8E4F0E080E197E2918352
:104950008083EEE4F0E080E88083EEE4F0E083E042
:104960008083A9E5B0E0E9E5F0E0808184608C9384
:10497000A5E5B0E0E5E5F0E080818A608C93ABE5E9
:10498000B0E0EBE5F0E08081806C8C93DF91CF911B
:104990000895CF93DF93CDB7DEB7E6E2F0E0108263
:1049A000E7E2F0E082E08083E8E2F0E080E8808304
:1049B000E6E2F0E085EE8083E0E5F0E01082EAE3F5
:1049C000F0E01082EBE3F0E01082DF91CF910895E8
:1049D000CF93DF93CDB7DEB7EAE2F0E088E98083DA
:1049E000E9E2F0E08FE0808382EC93E090938E0325
:1049F00080938D0380918D0390918E0390938A0311
:104A00008093890380E993E090938C0380938B03D8
:104A100080918B0390918C039093F5038093F40322
:104A200010928F0310925603DF91CF9108951F9239
:104A30000F920FB60F9211242F933F938F939F9352
:104A4000AF93BF93EF93FF93CF93DF93CDB7DEB7D1
:104A500080918F03882381F1ACE2B0E0E0918D0377
:104A6000F0918E0380818C9380918D0390918E03C1
:104A7000019690938E0380938D0320918D03309146
:104A80008E0384EF93E02817390730F082EC93E02F
:104A900090938E0380938D0380918F038150809338
:104AA0008F0380918F03882339F4AAE2B0E0EAE211
:104AB000F0E080818F7D8C93DF91CF91FF91EF911A
:104AC000BF91AF919F918F913F912F910F900FBE0A
:104AD0000F901F9018951F920F920FB60F921124EE
:104AE0002F933F938F939F93AF93BF93EF93FF9336
:104AF000CF93DF93CDB7DEB7A091F403B091F50368
:104B0000ECE2F0E080818C93809156038F5F80937C
:104B100056038091F4039091F50301969093F50369
:104B20008093F4032091F4033091F50382EC93E039
:104B30002817390730F080E993E09093F5038093CC
:104B4000F403DF91CF91FF91EF91BF91AF919F91CE
:104B50008F913F912F910F900FBE0F901F9018953E
:104B6000CF93DF93CDB7DEB723970FB6F894DEBFB0
:104B70000FBECDBF80915603882359F1F8948091E0
:104B80005603815080935603E0918B03F0918C0380
:104B90008081898380918B0390918C0301969093FF
:104BA0008C0380938B0320918B0330918C0382ECD8
:104BB00093E02817390730F080E993E090938C0355
:104BC00080938B0378948981282F33273B832A8312
:104BD00004C08FEF9FEF9B838A838A819B812396FA
:104BE0000FB6F894DEBF0FBECDBFDF91CF91089511
:104BF000CF93DF93CDB7DEB723970FB6F894DEBF20
:104C00000FBECDBF898380918F03823388F5F894DE
:104C100080918F038F5F80938F03E0918903F091E0
:104C20008A03898180838091890390918A03019608
:104C300090938A03809389032091890330918A039A
:104C400084EF93E02817390730F082EC93E09093DB
:104C50008A0380938903AAE2B0E0EAE2F0E080816F
:104C600080628C93789481E090E09B838A8302C079
:104C70001B821A828A819B8123960FB6F894DEBF2D
:104C80000FBECDBFDF91CF910895CF93DF93CDB706
:104C9000DEB724970FB6F894DEBF0FBECDBF9C835E
:104CA0008B838B819C819A8389830CC0E981FA81F3
:104CB00080810E94F825882329F089819A810196B4
:104CC0009A838983E981FA818081882379F781E059
:104CD00090E024960FB6F894DEBF0FBECDBFDF91F3
:104CE000CF910895CF93DF93CDB7DEB787E391E0FF
:104CF0000E944526DF91CF910895CF93DF93CDB7E2
:104D0000DEB7809156039927DF91CF910895CF9315
:104D1000DF93CDB7DEB765970FB6F894DEBF0FBE51
:104D2000CDBF9E878D876F87488BAE014C5F5F4FED
:104D30005A8B498B8AE391E09C8B8B8B99E09D8BFE
:104D4000EB89FC8900804B895C894F5F5F4F5C8BEE
:104D50004B8BE989FA89008249895A894F5F5F4FF5
:104D60005A8B498B5D8951505D8B8D89882341F722
:104D70001B8289E08A838AE089838F858823D1F02A
:104D80008A81282F332789E090E0FC01E21BF30B96
:104D90009F018F8599272817390760F08A818150F4
:104DA0008A838A819927FE013496E80FF91F8EE2E3
:104DB00080831F868A8181508A838A819927FE0198
:104DC0003496E80FF91F8981282F33278D859E851A
:104DD000B9010E94D53C805D80838981282F3327CB
:104DE0008D859E85B9010E94D53CCB019E878D871C
:104DF0008D859E85009719F48F85882321F08F85F6
:104E0000863008F4BACF8889893010F4888989837C
:104E100089E09889891B8A830EC08A81282F3327CD
:104E2000CE010496FC01E20FF31F80810E94F82559
:104E30008A818F5F8A838A81893078F365960FB67D
:104E4000F894DEBF0FBECDBFDF91CF910895CF9311
:104E5000DF93CDB7DEB722970FB6F894DEBF0FBE53
:104E6000CDBF9A838983E981FA81208189819A81E2
:104E700001969A838983822F0E94F825E981FA811D
:104E8000208189819A8101969A838983822F0E9449
:104E9000F825E981FA81208189819A8101969A8396
:104EA0008983822F0E94F825E981FA8180810E94FE
:104EB000F82522960FB6F894DEBF0FBECDBFDF9166
:104EC000CF910895CF93DF93CDB7DEB723970FB679
:104ED000F894DEBF0FBECDBF8B838B818823A1F0FA
:104EE0000DC01A82198205C089819A8101969A8320
:104EF000898389819A8189349105B0F38B818150AE
:104F00008B838B818F3F69F723960FB6F894DEBFB2
:104F10000FBECDBFDF91CF910895CF93DF93CDB773
:104F2000DEB723970FB6F894DEBF0FBECDBF8B83DD
:104F30008B818823A9F00EC01A82198205C089814D
:104F40009A8101969A83898389819A8122E08B3B99
:104F50009207A8F38B8181508B838B818F3F61F700
:104F600023960FB6F894DEBF0FBECDBFDF91CF9171
:104F70000895CF93DF93CDB7DEB723970FB6F8949C
:104F8000DEBF0FBECDBF8B838B818823A9F00EC0FF
:104F90001A82198205C089819A8101969A83898330
:104FA00089819A812BE18F349207A8F38B818150FC
:104FB0008B838B818F3F61F723960FB6F894DEBF0A
:104FC0000FBECDBFDF91CF910895CF93DF93CDB7C3
:104FD000DEB72E970FB6F894DEBF0FBECDBF9E870B
:104FE0008D872D853E85CE0109969A8389833C83E2
:104FF0002B8384E090E09E838D838D819E819887B2
:105000008F83AB81BC81E981FA818F81988501977B
:1050100024F00E941E3D0192FACFBC83AB83FA8339
:10502000E98398878F8389859A85AB85BC85BC0188
:10503000CD012E960FB6F894DEBF0FBECDBFDF9127
:10504000CF910895CF93DF93CDB7DEB764970FB6B6
:10505000F894DEBF0FBECDBF9A8B898B7C8B6B8B98
:105060008B899C89988B8F8789899A899E878D8760
:10507000ED85FE8540818D859E8501969E878D8775
:105080002F8538898F8598890196988B8F873B87E4
:105090002A874C878C85AA85BB85082E0E94263DD1
:1050A000BB87AA87ED85FE8540818D859E8501960B
:1050B0009E878D872F8538898F8598890196988B53
:1050C0008F8738872F8349878985AF81B885082ED8
:1050D0000E94263DB887AF83ED85FE8540818D8592
:1050E0009E8501969E878D872F8538898F85988923
:1050F0000196988B8F873D832C834E838E81AC8164
:10510000BD81082E0E94263DBD83AC83ED85FE85C2
:1051100040818D859E8501969E878D872F85388954
:105120008F8598890196988B8F873A8329834B8343
:105130008B81A981BA81082E0E94263DBA83A9835A
:1051400064960FB6F894DEBF0FBECDBFDF91CF914E
:1051500008956F927F928F929F92AF92BF92CF925B
:10516000DF92EF92FF920F931F93CF93DF93CDB710
:10517000DEB76A970FB6F894DEBF0FBECDBF9A8F29
:10518000898FE98DFA8D81E08083E98DFA8D148213
:10519000E98DFA8D80E090E0A0E4BFE384879587F5
:1051A000A687B787E98DFA8D8DEC9CECACECBEE35D
:1051B000808B918BA28BB38BE98DFA8D80E090E090
:1051C000A0E0B0E0848B958BA68BB78BE98DFA8D30
:1051D00080E090E0A0E0B0E0808F918FA28FB38F4D
:1051E000E98DFA8D80E090E0A0E8BFE3848F958F91
:1051F000A68FB78FE98DFA8D80E090E0A0E8B0E44B
:1052000080A391A3A2A3B3A3E98DFA8D83E393E3D3
:10521000A3E3BFE384A395A3A6A3B7A3E98DFA8D67
:1052200080E090E0A0EFB1E480A791A7A2A7B3A788
:10523000E98DFA8D80E090E0ACE8B2E484A795A710
:10524000A6A7B7A7E98DFA8D80E090E0A0E2B2E4CE
:1052500080AB91ABA2ABB3ABE98DFA8D80E090E06F
:10526000A0EAB0E484AB95ABA6ABB7ABE98DFA8D01
:1052700080E090E0A0E0B0E080AF91AFA2AFB3AF2C
:10528000E98DFA8D80E090E0A0E0B0E084AF95AFCA
:10529000A6AFB7AF898D9A8DFC01E05CFF4F80E02F
:1052A00090E0A0E8BEE380839183A283B383E98D7D
:1052B000FA8D2089318942895389898D9A8DFC0123
:1052C000EC58FF4F2083318342835383898D9A8D1D
:1052D000FC01E85BFF4F80E090E0A0E0B0E080835D
:1052E0009183A283B383898D9A8DFC01E45AFF4F89
:1052F00080E090E0A0E0B0E080839183A283B3835C
:10530000898D9A8DFC01E258FF4F8081918104962E
:105310009F8B8E8BAE89BF890E941E3D802DBF8BD7
:10532000AE8B888F888D9927E98DFA8D8483E98DDE
:10533000FA8D8481853038F0E98DFA8D1482898D5B
:105340009A8D0E942D31898D9A8DFC01E258FF4F74
:10535000808191819C8B8B8BAB89BC890E941E3D87
:10536000802DBC8BAB8B8D8B8D899927E98DFA8D28
:105370008083898D9A8DFC01E258FF4F8081918155
:105380000196998B888BA889B9890E941E3D802D32
:10539000B98BA88B8A8B8A899927E98DFA8D8183AD
:1053A000898D9A8DFC01E258FF4F80819181029690
:1053B0009E878D87AD85BE850E941E3D802DBE8750
:1053C000AD878F878F859927E98DFA8D8283898DA7
:1053D0009A8DFC01E258FF4F8081918103969B8753
:1053E0008A87AA85BB850E941E3D802DBB87AA8720
:1053F0008C878C859927E98DFA8D8383898D9A8D89
:10540000FC01E258FF4F80819181049698878F8339
:10541000AF81B8850E941E3D802DB887AF838987F4
:1054200089859927E98DFA8D8483898D9A8DFC0170
:10543000E258FF4F8081918105969D838C83AC81DA
:10544000BD810E941E3D802DBD83AC838E838E81E5
:105450009927E98DFA8D8583E98DFA8D1082E98D82
:10546000FA8D1082E98DFA8D81E08083E98DFA8DC5
:105470008481882329F0E98DFA8D81E0848303C03B
:10548000E98DFA8D1482E98DFA8D1482898D9A8DB9
:10549000FC01E258FF4F8081918106969A838983AF
:1054A000A981BA810E941E3D802DBA83A9838B8376
:1054B0008B819927E98DFA8D8683898D9A8DFC01E0
:1054C000E258FF4F8081918108960E94E527DC0118
:1054D000CB01E98DFA8D80AB91ABA2ABB3AB898DDB
:1054E0009A8DFC01E258FF4F808191810C960E94B9
:1054F000E527DC01CB01E98DFA8D80879187A287B2
:10550000B387898D9A8DFC01E258FF4F808191818C
:1055100040960E94E527DC01CB01E98DFA8D848756
:105520009587A687B787E98DFA8D248535854685C9
:105530005785898D9A8DFC01E059FF4F2083318377
:1055400042835383898D9A8DFC01E258FF4F8081FD
:10555000918144960E94E527DC01CB01E98DFA8D0B
:10556000808B918BA28BB38B898D9A8DFC01E25835
:10557000FF4F8081918148960E94E527DC01CB0195
:10558000E98DFA8D848B958BA68BB78B898D9A8D3F
:10559000FC01E258FF4F808191814C960E94E527E3
:1055A000DC01CB01E98DFA8D808F918FA28FB38FB3
:1055B000898D9A8DFC01E258FF4F80819181809600
:1055C0000E94E5279B01AC01898D9A8DFC01EC5866
:1055D000FF4F2083318342835383898D9A8DFC0151
:1055E000E258FF4F8081918184960E94E527DC017B
:1055F000CB01E98DFA8D80A391A3A2A3B3A3898DDA
:105600009A8DFC01E258FF4F8081918188960E941B
:10561000E527DC01CB01E98DFA8D84A395A3A6A330
:10562000B7A3898D9A8DFC01E258FF4F808191814B
:105630008C960E94E527DC01CB01E98DFA8D80A7CD
:1056400091A7A2A7B3A7898D9A8DFC01E258FF4FBD
:1056500080819181C0960E94E527DC01CB01E98D14
:10566000FA8D84A795A7A6A7B7A7898D9A8DFC0167
:10567000E258FF4F80819181C4960E94E527DC01AA
:10568000CB01E98DFA8D84AB95ABA6ABB7AB898D19
:105690009A8DFC01E258FF4F80819181C8960E944B
:1056A000E5279B01AC01898D9A8DFC01E05CFF4FE1
:1056B0002083318342835383EFE3F0E01082EEE3F3
:1056C000F0E01082898D9A8DFC01E05CFF4F8081B3
:1056D0009181A281B3812FE632E143E85AE3BC0114
:1056E000CD010E94FE3B88230CF00DC0898D9A8D60
:1056F000FC01E05CFF4F8FE692E1A3E8BAE3808310
:105700009183A283B383E98DFA8D80899189A289DF
:10571000B38920E030E040E050E0BC01CD010E94C0
:10572000FE3B18160CF40AC0E98DFA8D80E090E07B
:10573000A0E2B1E4808B918BA28BB38B898D9A8D83
:10574000FC01EC58FF4F80819181A281B38120E060
:1057500030E040E050E0BC01CD010E94FE3B181655
:105760000CF40DC0898D9A8DFC01EC58FF4F80E040
:1057700090E0A0E2B1E480839183A283B383898D1A
:105780009A8DFC01E05CFF4F80819181A281B38101
:1057900020E030E040E050E0BC01CD010E94FE3B43
:1057A00018160CF40DC0898D9A8DFC01E05CFF4F3A
:1057B00080E090E0A0E8BFE380839183A283B3837D
:1057C000E98DFA8D80A191A1A2A1B3A120E030E0E2
:1057D00040E050E0BC01CD010E94FE3B18160CF4E5
:1057E0000AC0E98DFA8D80E090E0A0E2B1E480A3E8
:1057F00091A3A2A3B3A3E98DFA8D84A995A9A6A923
:10580000B7A920E030E040E050E0BC01CD010E94AB
:10581000FE3B18160CF40AC0E98DFA8D80E090E08A
:10582000A0E2B1E484AB95ABA6ABB7ABE98DFA8D42
:10583000E484F58406851785898D9A8DFC01E05CEA
:10584000FF4F80819181A281B3819C01AD01C8018C
:10585000B7010E946E3CDC01CB017C018D01E98D1A
:10586000FA8D80899189A289B3899C01AD01C80113
:10587000B7010E94913BDC01CB019C01AD01898DF8
:105880009A8DFC01E05AFF4F20833183428353837A
:10589000898D9A8DFC01E05CFF4FE080F1800281F0
:1058A0001381898D9A8DFC01EC58FF4F8081918185
:1058B000A281B3819C01AD01C801B7010E94913B57
:1058C000DC01CB019C01AD01898D9A8DFC01EC5965
:1058D000FF4F2083318342835383E98DFA8DE48423
:1058E000F58406851785E98DFA8D80A191A1A2A185
:1058F000B3A19C01AD01C801B7010E946E3CDC015F
:10590000CB017C018D01E98DFA8D84899589A68969
:10591000B7899C01AD01C801B7010E946E3CDC0152
:10592000CB013C014D01E98DFA8DA488B588C6886C
:10593000D788E98DFA8DE0A0F1A002A113A1898D8D
:105940009A8DFC01E05CFF4F80819181A281B3813F
:105950009C01AD01C801B7010E946E3CDC01CB0186
:105960009C01AD01C601B5010E944F3BDC01CB019A
:105970009C01AD01C401B3010E94913BDC01CB014C
:105980009C01AD01898D9A8DFC01E859FF4F208360
:10599000318342835383E98DFA8D648875888688C4
:1059A0009788E98DFA8DA488B588C688D788E98D4F
:1059B000FA8DE0A0F1A002A113A1898D9A8DFC01BE
:1059C000E05CFF4F80819181A281B3819C01AD0198
:1059D000C801B7010E946E3CDC01CB019C01AD0106
:1059E000C601B5010E944F3BDC01CB019C01AD011A
:1059F000C401B3010E94913BDC01CB019C01AD01CC
:105A0000898D9A8DFC01E459FF4F208331834283B5
:105A100053836A960FB6F894DEBF0FBECDBFDF91F9
:105A2000CF911F910F91FF90EF90DF90CF90BF909B
:105A3000AF909F908F907F906F9008956F927F921C
:105A40008F929F92AF92BF92CF92DF92EF92FF928E
:105A50000F931F93CF93DF93CDB7DEB722970FB687
:105A6000F894DEBF0FBECDBF9A838983E981FA81A6
:105A7000E484F5840685178589819A81FC01E059C3
:105A8000FF4F80819181A281B3819C01AD01C8014A
:105A9000B7010E944E3BDC01CB0120E030E040E04A
:105AA00050E0BC01CD010E94FE3B882309F461C097
:105AB00089819A81FC01E85BFF4F60807180828060
:105AC0009380E981FA81E484F584068517858981CC
:105AD0009A81FC01E059FF4F80819181A281B381BD
:105AE0009C01AD01C801B7010E944E3BDC01CB0116
:105AF0005C016D01E981FA81E4A0F5A006A117A17E
:105B0000E981FA8180859185A285B3859C01AD01EB
:105B1000C801B7010E946E3CDC01CB017C018D0104
:105B2000E981FA8180AD91ADA2ADB3AD9C01AD012B
:105B3000C801B7010E944E3BDC01CB019C01AD01C5
:105B4000C601B5010E946E3CDC01CB019C01AD0198
:105B5000C401B3010E944E3BDC01CB019C01AD01AD
:105B600089819A81FC01E85BFF4F20833183428366
:105B70005383E981FA81A484B584C684D784E981FA
:105B8000FA81E4A0F5A006A117A1E981FA81808538
:105B90009185A285B3859C01AD01C801B7010E9422
:105BA0006E3CDC01CB017C018D01E981FA8180AD85
:105BB00091ADA2ADB3AD9C01AD01C801B7010E948A
:105BC0004E3BDC01CB019C01AD01C601B5010E9439
:105BD0006E3CDC01CB019C01AD0189819A81FC0105
:105BE000EC5BFF4F208331834283538389819A8109
:105BF000FC01E459FF4FE080F1800281138189812B
:105C00009A81FC01E45BFF4F80819181A281B38185
:105C10009C01AD01C801B7010E946E3CDC01CB01C3
:105C20003C014D0189819A81FC01E859FF4FA08018
:105C3000B180C280D380E981FA81E0ACF1AC02ADE1
:105C400013AD89819A81FC01E45AFF4F80819181D3
:105C5000A281B3819C01AD01C801B7010E944E3BF6
:105C6000DC01CB019C01AD01C601B5010E946E3C77
:105C7000DC01CB019C01AD01C401B3010E944E3B8C
:105C8000DC01CB019C01AD0189819A81FC01E45BBF
:105C9000FF4F208331834283538389819A81FC01A2
:105CA000EC5BFF4FE080F1800281138189819A8152
:105CB000FC01E85BFF4F80819181A281B3819C014F
:105CC000AD01C801B7010E944F3BDC01CB017C0153
:105CD0008D0189819A81FC01E45BFF4F8081918174
:105CE000A281B3819C01AD01C801B7010E944F3B65
:105CF000DC01CB019C01AD0189819A81FC01E85A4C
:105D0000FF4F2083318342835383E981FA8180816D
:105D1000882309F476C089819A81FC01E85BFF4FF2
:105D2000608071808280938089819A81FC01E05A31
:105D3000FF4FA080B180C280D380E981FA81E084E6
:105D4000F18402851385E981FA8180AD91ADA2AD20
:105D5000B3AD9C01AD01C801B7010E944E3BDC010F
:105D6000CB019C01AD01C601B5010E946E3CDC0176
:105D7000CB019C01AD01C401B3010E944F3BDC018A
:105D8000CB013C014D0189819A81FC01EC59FF4F07
:105D9000A080B180C280D38089819A81FC01EC5AB5
:105DA000FF4FE080F1800281138189819A81FC019B
:105DB000E85AFF4F80819181A281B3819C01AD019E
:105DC000C801B7010E944E3BDC01CB019C01AD0133
:105DD000C601B5010E946E3CDC01CB019C01AD0106
:105DE000C401B3010E944F3BDC01CB019C01AD011A
:105DF00089819A81FC01E85BFF4F208331834283D4
:105E00005383E981FA818481813009F0A8C08981B6
:105E10009A81FC01E85AFF4F80819181A281B38170
:105E20009C01AD0160E070E088EC92E40E944E3B82
:105E3000DC01CB017C018D01E981FA8180A591A56E
:105E4000A2A5B3A59C01AD01C801B7010E94FE3B0C
:105E500088230CF010C0E981FA8120A531A542A564
:105E600053A589819A81FC01EC5AFF4F208331832D
:105E70004283538352C089819A81FC01E85AFF4FC3
:105E800080819181A281B3819C01AD0160E070E0CD
:105E900088EC92E40E944E3BDC01CB017C018D0139
:105EA000E981FA8184A595A5A6A5B7A59C01AD01B8
:105EB000C801B7010E94013C18160CF010C0E9811E
:105EC000FA8124A535A546A557A589819A81FC01AB
:105ED000EC5AFF4F20833183428353831EC0898154
:105EE0009A81FC01E85AFF4F80819181A281B381A0
:105EF0009C01AD0160E070E088EC92E40E944E3BB2
:105F0000DC01CB019C01AD0189819A81FC01EC5A35
:105F1000FF4F208331834283538389819A81FC011F
:105F2000EC5AFF4F80819181A281B38126E636ED44
:105F300043E254E4BC01CD010E946E3CDC01CB0184
:105F4000BC01CD010E94D73BDC01CB019C018981C2
:105F50009A81FC01E458FF4F3183208383C08981FB
:105F60009A81FC01E85AFF4FE080F18002811381A1
:105F7000E981FA8180A591A5A2A5B3A59C01AD01F7
:105F8000C801B7010E94FE3B88230CF010C0E981D4
:105F9000FA8120A531A542A553A589819A81FC01EA
:105FA000EC5AFF4F20833183428353833AC0898167
:105FB0009A81FC01E85AFF4FE080F1800281138151
:105FC000E981FA8184A595A5A6A5B7A59C01AD0197
:105FD000C801B7010E94013C18160CF010C0E981FD
:105FE000FA8124A535A546A557A589819A81FC018A
:105FF000EC5AFF4F208331834283538312C089813F
:106000009A81FC01E85AFF4F2081318142815381FE
:1060100089819A81FC01EC5AFF4F208331834283AE
:10602000538389819A81FC01EC5AFF4F80819181D1
:10603000A281B38120E030E04BE154E4BC01CD010A
:106040000E946E3CDC01CB01BC01CD010E94D73B1C
:10605000DC01CB019C0189819A81FC01E458FF4F4E
:1060600031832083E981FA8120AD31AD42AD53AD5A
:1060700089819A81FC01E45AFF4F20833183428356
:106080005383E981FA812485358546855785898141
:106090009A81FC01E059FF4F20833183428353836F
:1060A000E981FA81818122960FB6F894DEBF0FBE96
:1060B000CDBFDF91CF911F910F91FF90EF90DF90B7
:1060C000CF90BF90AF909F908F907F906F900895EA
:1060D000CF93DF93CDB7DEB722970FB6F894DEBF2C
:1060E0000FBECDBF9A83898382E80E94F82588E598
:1060F0000E94F825E981FA818081880F0E94F825A5
:10610000E981FA8181810E94F825E981FA81828101
:106110000E94F825E981FA8183810E94F825E981AE
:10612000FA8184810E94F825E981FA8185810E94A3
:10613000F825E981FA8186810E94F82580E00E9495
:10614000F82582E00E94B92789819A81C0960E9431
:10615000272789819A8108960E94272789819A8119
:106160000C960E94272782E00E94B92789819A8194
:1061700040960E94272789819A8144960E9427276A
:1061800089819A8148960E94272782E00E94B92738
:1061900089819A818C589F4F0E94272789819A81F3
:1061A00080960E94272789819A8184960E942727BA
:1061B00082E00E94B92789819A8188960E942727C8
:1061C00089819A818C960E94272789819A81C49619
:1061D0000E94272782E00E94B92789819A81CC9664
:1061E0000E94272789819A81C8960E942727898142
:1061F0009A81805C9F4F0E94272782E00E94B927E6
:1062000089819A818C5B9F4F0E94272789819A817F
:10621000885B9F4F0E94272789819A81845B9F4FCB
:106220000E94272782E00E94B92789819A818C5990
:106230009F4F0E94272789819A818C5A9F4F0E94E5
:1062400027278DE70E94F82522960FB6F894DEBF27
:106250000FBECDBFDF91CF910895CF93DF93CDB720
:10626000DEB72E970FB6F894DEBF0FBECDBF9E8768
:106270008D87ED85FE8520818D859E85FC01E25808
:10628000FF4F808191819B878A872C878C85AA8587
:10629000BB85082E0E94263DBB87AA87ED85FE851B
:1062A00021818D859E85FC01E258FF4F808191817F
:1062B000019698878F8329878985AF81B885082EB5
:1062C0000E94263DB887AF83ED85FE8524818D85AC
:1062D0009E85FC01E258FF4F8081918104969D8349
:1062E0008C832E838E81AC81BD81082E0E94263D39
:1062F000BD83AC83ED85FE8525818D859E85FC0162
:10630000E258FF4F8081918105969A8389832B8380
:106310008B81A981BA81082E0E94263DBA83A98368
:106320008D859E85FC01E258FF4F80819181089602
:106330009C018D859E85C096B9010E9422288D857D
:106340009E85FC01E258FF4F808191810C969C0153
:106350008D859E850896B9010E9422288D859E858F
:10636000FC01E258FF4F8081918140969C018D8510
:106370009E850C96B9010E9422288D859E85FC0180
:10638000E258FF4F8081918144969C018D859E85C6
:106390004096B9010E9422288D859E85FC01E25815
:1063A000FF4F8081918148969C018D859E85449602
:1063B000B9010E9422288D859E85FC01E258FF4F7D
:1063C000808191814C969C018D859E854896B9016E
:1063D0000E9422288D859E85FC01E258FF4F808116
:1063E000918180969C018D859E858C589F4FB90127
:1063F0000E9422288D859E85FC01E258FF4F8081F6
:10640000918184969C018D859E858096B9010E941C
:1064100022288D859E85FC01E258FF4F8081918165
:1064200088969C018D859E858496B9010E942228BC
:106430008D859E85FC01E258FF4F808191818C966D
:106440009C018D859E858896B9010E9422288D85A4
:106450009E85FC01E258FF4F80819181C0969C018E
:106460008D859E858C96B9010E9422288D859E85FA
:10647000FC01E258FF4F80819181C4969C018D857B
:106480009E85C496B9010E9422288D859E85FC01B7
:10649000E258FF4F80819181C8969C018D859E8531
:1064A000805C9F4FB9010E942228EFE3F0E0108248
:1064B000EEE3F0E010822E960FB6F894DEBF0FBE2A
:1064C000CDBFDF91CF910895CF93DF93CDB7DEB7E6
:1064D0002C970FB6F894DEBF0FBECDBF1A86198673
:1064E00018861F82A8958091F603282F33273C87B2
:1064F0002B878B859C858838910509F4E2C02B8514
:106500003C852938310554F58B859C85803891056B
:1065100009F416C22B853C85213831056CF48B8536
:106520009C858333910509F496C32B853C852433E0
:10653000310509F493C3A5C38B859C8583389105E8
:1065400009F41AC22B853C852538310509F441C070
:106550008B859C858138910561F193C32B853C85A2
:106560002339310509F49AC38B859C8584399105BB
:106570006CF42B853C852A38310509F472C08B8573
:106580009C858139910509F419C17BC32B853C8514
:106590002839310509F452C18B859C8589399105CB
:1065A00009F461C32B853C852539310509F491C176
:1065B00068C382E08093F60380917A0199279695CB
:1065C000982F882797958795805B9D4F0E9468300C
:1065D00065C38091F803282F33278091F903992709
:1065E000982F8827820F931F98878F831A86198682
:1065F00021C0A89589859A850296FC01E850FC4F38
:1066000040812F81388589859A85820F931F9D83CC
:106610008C834E838E81AC81BD81082E0E94263DE5
:10662000BD83AC8382E00E948D2789859A8501967F
:106630009A8789878091F703992702979C0189851A
:106640009A8582179307A8F286E80E94F82581E0D0
:106650000E94F82581E00E94F82589E70E94F8252C
:106660001DC38091F803282F33278091F9039927C0
:10667000982F8827820F931F98878F838BE80E941B
:10668000F82583E00E94F8258F8198859A83898375
:10669000A981BA810E941E3D802DBA83A9838B8374
:1066A0008B8199270E94F8258F810E94F8258F8180
:1066B0009885892F99270E94F82584E70E94F8255C
:1066C000EDC289E80E94F82580E10E94F8258091BA
:1066D0008301909184010E94F8258091830190911B
:1066E0008401892F99270E94F82580918501909136
:1066F00086010E94F8258091850190918601892F5D
:1067000099270E94F82580918701909188010E9425
:10671000F8258091870190918801892F99270E94FF
:10672000F8258091890190918A010E94F825809135
:10673000890190918A01892F99270E94F82583E089
:106740000E948D2780918B0190918C010E94F825E9
:1067500080918B0190918C01892F99270E94F825B7
:1067600080918D0190918E010E94F82580918D017C
:1067700090918E01892F99270E94F82580918F0191
:10678000909190010E94F82580918F019091900145
:10679000892F99270E94F82580919101909192016B
:1067A0000E94F8258091910190919201892F99275B
:1067B0000E94F82586E70E94F82570C282E90E94AF
:1067C000F82580E10E94F82580917A019927969515
:1067D000982F8827979587958C5A9F4F805B9D4F60
:1067E0000E94272780917A0199279695982F8827CC
:1067F00097958795C896805B9D4F0E94272780912B
:106800007A0199279695982F8827979587950896C6
:10681000805B9D4F0E94272780917A01992796954A
:10682000982F882797958795885B9F4F805B9D4F12
:106830000E9427278DE60E94F82530C287E90E9432
:10684000F8258EE00E94F82588E093E00E94272733
:1068500088E892E00E942727809187019091880123
:106860000E94F8258091870190918801892F9927AE
:106870000E94F825ECE5F0E0808199279C01220F29
:10688000331FC901880F991F880F991F820F931F0B
:10689000C29729E130E0B9010E94E93CCB010E9496
:1068A000F82580918501909186010E94F8258091BC
:1068B0009701909198010E94F825809197019091FD
:1068C0009801892F99270E94F82588E60E94F825CB
:1068D000E5C186E90E94F82580E10E94F8258091B3
:1068E0007A0199279695982F8827979587958C5A9E
:1068F0009F4F805B9D4F0E9427278BEC91E00E9469
:10690000272780917A0199279695982F8827979520
:1069100087950896805B9D4F0E94272780917A017A
:1069200099279695982F882797958795885B9F4FED
:10693000805B9D4F0E94272789E60E94F825AEC103
:106940008091F80380937A0180917A01882331F055
:1069500080917A01813011F010927A0180E80E94D2
:10696000F82581E00E94F82580917A010E94F8259F
:106970008FE70E94F82592C184E80E94F82584E2FE
:106980000E94F82580916000909161000E94F82596
:106990008091600090916100892F99270E94F825CD
:1069A00080916200909163000E94F82580916200BE
:1069B00090916300892F99270E94F82585E00E9415
:1069C0008D2780916400909165000E94F825809148
:1069D000640090916500892F99270E94F825809185
:1069E0008200909183002AE030E0B9010E94D53CFA
:1069F000CB010E94F82580918200909183002AE0CB
:106A000030E0B9010E94D53CCB01892F99270E9423
:106A1000F82580916600909167002AE030E0B90186
:106A20000E94D53CCB010E94F82580916600909190
:106A300067002AE030E0B9010E94D53CCB01892FE4
:106A400099270E94F82580916800909169002AE0BA
:106A500030E0B9010E94D53CCB010E94F82585E0C9
:106A60000E948D2780916800909169002AE030E0B3
:106A7000B9010E94D53CCB01892F99270E94F825A6
:106A800080916A0090916B002AE030E0B9010E9489
:106A9000D53CCB010E94F82580916A0090916B0053
:106AA0002AE030E0B9010E94D53CCB01892F99271B
:106AB0000E94F82580916E0090916F002AE030E0EE
:106AC000B9010E94D53CCB010E94F82580916E004F
:106AD00090916F002AE030E0B9010E94D53CCB01D3
:106AE000892F99270E94F82580919B0090919C0006
:106AF0000E94F82580919B0090919C00892F9927F6
:106B00000E94F82585E00E948D2780917000909169
:106B100071002AE030E0B9010E94D53CCB010E940F
:106B2000F82580917000909171002AE030E0B90161
:106B30000E94D53CCB01892F99270E94F82580918E
:106B40008400909185002AE030E0B9010E94D53C94
:106B5000CB010E94F82580918400909185002AE065
:106B600030E0B9010E94D53CCB01892F99270E94C2
:106B7000F82580917200909173000E94F825809111
:106B8000720090917300892F99270E94F82585E063
:106B90000E948D27809176000E94F82580917700D1
:106BA0000E94F825809178000E94F8258091790054
:106BB0000E94F82580917A000E94F82580917B0040
:106BC0000E94F82585E00E948D2780917C0090919D
:106BD0007D002AE030E0B9010E94D53CCB010E9443
:106BE000F82580917C0090917D002AE030E0B90189
:106BF0000E94D53CCB01892F99270E94F8258091CE
:106C00007E0090917F002AE030E0B9010E94D53CDF
:106C1000CB010E94F82580917E0090917F002AE0B0
:106C200030E0B9010E94D53CCB01892F99270E9401
:106C3000F82580918000909181000E94F825809134
:106C4000800090918100892F99270E94F8258BE779
:106C50000E94F82523C00E94FC2020C00E94A81B8F
:106C60000E942A171BC0F89488E190E028E00FB634
:106C7000F894A89581BD0FBE21BD88EC0E94B9276C
:106C80000DC08EE80E94F82581E00E94F8258091D1
:106C9000F6030E94F82581E70E94F8251092F6037A
:106CA0001A8619860BC089859A85FC01E850FC4F2D
:106CB000108289859A8501969A8789878091F70342
:106CC000282F332789859A858217930760F31092BE
:106CD000F7032C960FB6F894DEBF0FBECDBFDF9141
:106CE000CF910895CF93DF93CDB7DEB724970FB63A
:106CF000F894DEBF0FBECDBF9B838A836C8319825D
:106D000088E190E02DE00FB6F894A89581BD0FBE04
:106D100021BDE9C080914D02882309F07CC08981A2
:106D200099279C018A819B81F901E80FF91F8081D5
:106D30008093F6038091F603833309F45AC080915F
:106D4000F603843309F455C08091F603883509F4BD
:106D500050C08091F603813609F44BC08091F60350
:106D6000853609F446C08091F6038F3609F441C098
:106D70008091F603803709F43CC08091F603873791
:106D8000C1F18091F6038937A1F18091F603803833
:106D900081F18091F6038A3761F18091F6038138A1
:106DA00041F18091F603833821F18091F603843814
:106DB00001F18091F6038538E1F08091F60388387F
:106DC000C1F08091F6038A38A1F08091F6038139F1
:106DD00081F08091F603833961F08091F603853963
:106DE00041F08091F603883921F08091F6038939CA
:106DF00021F481E080934D0273C08FE80E94F82552
:106E000081E00E94F8258091F6030E94F82580E732
:106E10000E94F82565C080914D028130A9F48981D6
:106E200099279C018A819B81F901E80FF91F8081D4
:106E30008093F7038091F703833310F010924D0293
:106E400082E080934D024CC080914D02282F332761
:106E50008091F7039927029628173907D1F480917A
:106E6000F603809580934D02898199279C018A8140
:106E70009B81F901E80FF91F908180914D029817CD
:106E800029F410924D020E9464322AC010924D02E1
:106E900027C080914D02823018F180914D02282F39
:106EA00033278091F7039927029628173907C4F4EE
:106EB00080914D029927AC01425050408981992719
:106EC0009C018A819B81F901E80FF91F8081FA01F9
:106ED000E850FC4F808380914D028F5F80934D027C
:106EE00089818F5F898399818C81981708F412CFEB
:106EF00024960FB6F894DEBF0FBECDBFDF91CF91C1
:106F00000895CF93DF93CDB7DEB70E9490370E94EC
:106F100012388BE591E00E947E38DF91CF91089581
:106F2000CF93DF93CDB7DEB7A4E3B0E0E4E3F0E0C6
:106F3000808180648C93A4E3B0E0E4E3F0E080819E
:106F400080618C93A4E3B0E0E4E3F0E080818062B0
:106F50008C9310922B04E5E3F0E0808180648083C1
:106F6000E5E3F0E08081806180838EE10E948D27DF
:106F700068EF81E00E94AB3882E00E948D2768EFC5
:106F800088E30E94AB3868EF8FE00E94AB3868EF6F
:106F900086E00E94AB3868EF81E00E94AB3882E067
:106FA0000E948D27DF91CF910895CF93DF93CDB7C6
:106FB000DEB768EF81E00E94AB3810924E0210926B
:106FC0004F02DF91CF910895CF93DF93CDB7DEB716
:106FD00068EF8BE30E94AB38DF91CF910895CF9398
:106FE000DF93CDB7DEB768EF88E30E94AB38DF915F
:106FF000CF910895CF93DF93CDB7DEB721970FB62A
:10700000F894DEBF0FBECDBF89836AEF89810E94ED
:10701000AB3821960FB6F894DEBF0FBECDBFDF911F
:10702000CF910895CF93DF93CDB7DEB710924E0284
:1070300080914F028F5F80934F0280914F02823088
:1070400010F010924F020E942838DF91CF910895DE
:10705000CF93DF93CDB7DEB780914F029927FC0124
:10706000E55BFE4F908180914E02890F68EF0E9490
:10707000AB38DF91CF910895CF93DF93CDB7DEB7D3
:1070800022970FB6F894DEBF0FBECDBF89836A8307
:10709000898180934E028A8180934F020E94283812
:1070A00022960FB6F894DEBF0FBECDBFDF91CF9111
:1070B0000895CF93DF93CDB7DEB721970FB6F8943D
:1070C000DEBF0FBECDBF898389818A3029F40E943B
:1070D00012380E94283809C06AEF89810E94AB38B3
:1070E00080914E028F5F80934E0221960FB6F894E6
:1070F000DEBF0FBECDBFDF91CF910895CF93DF9359
:10710000CDB7DEB724970FB6F894DEBF0FBECDBF64
:107110009A83898389819A819C838B83EB81FC810B
:10712000309781F00AC0EB81FC8180810E94593840
:107130008B819C8101969C838B83EB81FC81808178
:10714000882389F724960FB6F894DEBF0FBECDBF13
:10715000DF91CF910895CF93DF93CDB7DEB724971A
:107160000FB6F894DEBF0FBECDBF8B836C838C81CE
:107170008983000000000000000000000000000003
:1071800000000000000000000000000000000000FF
:1071900000008B81282F332780912E0490912F049B
:1071A000820F931F90932F0480932E0480912E04BE
:1071B00090912F0482959295907F9827807F9827B1
:1071C00090932F0480932E048B81282F3327809156
:1071D0002E0490912F04822B932B90932F04809355
:1071E0002E0480912E0490912F048F709F709093A5
:1071F0002F0480932E04E5E3F0E08081806180839A
:10720000E5E3F0E080818F7B808388E08A83E5E39B
:10721000F0E080818F7E8083E5E3F0E080818F7DE8
:1072200080838C81880F8C83A5E3B0E0EFE5F0E0EC
:10723000808181708170982F9295990F907E8C91AA
:107240008F7D892B8C93000000000000000000005F
:10725000000000000000000000000000000000002E
:10726000000000000000E5E3F0E0808180618083A1
:107270008A8181508A830000000000000000000025
:1072800000000000000000000000000000000000FE
:107290000000000000008A81882389F000000000BF
:1072A00000000000000000000000000000000000DE
:1072B000000000000000000000000000A8CF80E1F6
:1072C0008A83E5E3F0E080818F7E8083E5E3F0E070
:1072D00080818F7D808380912E0490912F049695DC
:1072E000879590932F0480932E04A5E3B0E0EFE5FB
:1072F000F0E0808181708170982F9295990F907E37
:107300008C918F7D892B8C93E5E3F0E08081806107
:1073100080838A8181508A83000000000000000081
:10732000000000000000000000000000000000005D
:10733000000000000000000000000000000000004D
:10734000000000000000000000000000000000003D
:10735000000000000000000000000000000000002D
:10736000000000000000000000000000000000001D
:1073700000000000000000008A81882309F0A1CFEE
:10738000E5E3F0E0808180648083E5E3F0E08081E4
:107390008061808389818A3F21F481E00E94622795
:1073A00003C082E00E948D2724960FB6F894DEBFBA
:1073B0000FBECDBFDF91CF910895CF93DF93CDB7AF
:1073C000DEB765970FB6F894DEBF0FBECDBF9E87C0
:1073D0008D876F87488BAE014C5F5F4F5A8B498B0F
:1073E00082E691E09C8B8B8B99E09D8BEB89FC89ED
:1073F00000804B895C894F5F5F4F5C8B4B8BE989C9
:10740000FA89008249895A894F5F5F4F5A8B498BAD
:107410005D8951505D8B8D89882341F71B8289E0FE
:107420008A838AE089838F858823D1F08A81282FF7
:10743000332789E090E0FC01E21BF30B9F018F856D
:1074400099272817390760F08A8181508A838A81B9
:107450009927FE013496E80FF91F8EE280831F867C
:107460008A8181508A838A819927FE013496E80FA8
:10747000F91F8981282F33278D859E85B9010E94A8
:10748000D53C805D80838981282F33278D859E851B
:10749000B9010E94D53CCB019E878D878D859E8545
:1074A000009719F48F85882321F08F85863008F4A2
:1074B000BACF8889893010F48889898389E09889CE
:1074C000891B8A830EC08A81282F3327CE01049618
:1074D000FC01E20FF31F80810E9459388A818F5F7F
:1074E0008A838A81893078F365960FB6F894DEBF77
:1074F0000FBECDBFDF91CF910895CF93DF93CDB76E
:10750000DEB765970FB6F894DEBF0FBECDBF9E877E
:107510008D876F87488BAE014C5F5F4F5A8B498BCD
:107520008BE691E09C8B8B8B99E09D8BEB89FC89A2
:1075300000804B895C894F5F5F4F5C8B4B8BE98987
:10754000FA89008249895A894F5F5F4F5A8B498B6C
:107550005D8951505D8B8D89882341F71B8289E0BD
:107560008A838AE089838D859E8599235CF48D8545
:107570009E85909581959F4F9E878D878DE28C8308
:1075800081E08B838F858823D1F08A81282F332750
:1075900089E090E0FC01E21BF30B9F018F859927A6
:1075A0002817390760F08A8181508A838A81992758
:1075B000FE013496E80FF91F8EE280831F868A81D0
:1075C00081508A838A819927FE013496E80FF91F3A
:1075D0008981282F33278D859E85B9010E94E93C3A
:1075E000805D80838981282F33278D859E85B90111
:1075F0000E94E93CCB019E878D878D859E850097F3
:1076000019F48F85882321F08F85863008F4BACF4E
:107610008B818130F9F488E0898319C08981282F12
:107620003327CE010496FC01E20FF31F80818032E4
:1076300059F48981282F3327CE010496FC01E20FEB
:10764000F31F8DE280831B828981815089838B8126
:10765000813021F38889893010F48889898389E011
:107660009889891B8A830EC08A81282F3327CE01EF
:107670000496FC01E20FF31F80810E9459388A8131
:107680008F5F8A838A81893078F365960FB6F89484
:10769000DEBF0FBECDBFDF91CF9108955058192E98
:1076A000EFD001D0D2C0BA176207730784079507DD
:1076B000B1F188F40EF410940B2EBA2FA02D062EE3
:1076C000622F202D072E732F302D082E842F402D52
:1076D000092E952F502DFF275523B9F0591B49F03E
:1076E000573E98F0469537952795A795F0405395C6
:1076F000C9F776F0BA0F621F731F841F30F48795A5
:1077000077956795B795F040939517FA0F2E0895E2
:10771000BF1BBB27BA0B620B730B840BF6CFDEF6D5
:10772000DBC0AED001D091C0552359F0992369F048
:107730009F575F57951B33F442F4903811F49158DA
:1077400005C09BC091589F3F09F4C6C0BB271124B8
:1077500062177307840730F4660F771F881FBB1FFB
:10776000915098F311D00F920FD00F920DD0A0E846
:107770002617370748071B0609F0A048BA2F602DC7
:107780007F918F9100240895A0E800246217730769
:107790008407B10528F0621B730B840BB1090A2A18
:1077A000660F771F881FBB1FA69581F7089597FB6B
:1077B00073D09F3738F0FEE9F91B982F872F762F6B
:1077C0006B2F05C086C09695879577956795F15084
:1077D000D0F73EF490958095709561957F4F8F4FCF
:1077E0009F4F0895E89403C097FB0EF4F3DFB62F84
:1077F000672F782F892F9EE9002427C00ED05EF0D6
:1078000004C00BD026F001C008D019F020F48FEF8F
:10781000089580E0089581E0089597FB092E0526DC
:1078200000F8689430D0E89407FC07C0621773072B
:107830008407950721F008F400940794989408951C
:107840009A95BB0F661F771F881F11249923A1F0FB
:107850008823B2F79F3F59F0BB0F48F421F4002072
:1078600011F460FF04C06F5F7F4F8F4F9F4F881FE1
:107870009795879597F908952CC09FEF80EC089510
:10788000052E092607FA440F551F5F3F79F0AA27F6
:10789000A51708F051E04795880F991F9F3F31F0D9
:1078A000BB27B91708F091E0879508959F919F91A4
:1078B0001124E3CF97FB880F991F9F3F31F0BB271F
:1078C000B91708F091E0879508959F919F91112431
:1078D000D4CF66277727882799270895D1DF01D04D
:1078E000B4CF992339F0552329F09F575F57950F4F
:1078F00013F49AF1F1CF91589F3FE1F3629FA12DCC
:107900000F92BB27639FA00DB11DEE27729FA00DA4
:10791000B11DEE1FAF93AA27649FB00DE11D739FA9
:10792000B00DE11DAA1F6627829FB00DE11DA61FA5
:107930005527749FE00DA11D551F839FE00DA11DCC
:10794000561F849FA00D511D852F7A2F6E2F1F90DB
:107950000F9088231AF4939539F48FCF000C111CE3
:10796000BB1F661F771F881F01280895629FD001E3
:10797000739FF001829FE00DF11D649FE00DF11DEA
:10798000929FF00D839FF00D749FF00D659FF00D99
:107990009927729FB00DE11DF91F639FB00DE11D86
:1079A000F91FBD01CF0111240895AA1BBB1B51E192
:1079B00007C0AA1FBB1FA617B70710F0A61BB70B5F
:1079C000881F991F5A95A9F780959095BC01CD0104
:1079D000089597FB092E07260AD077FD04D0E5DF2E
:1079E00006D000201AF4709561957F4F0895F6F740
:1079F000909581959F4F0895A1E21A2EAA1BBB1B5B
:107A0000FD010DC0AA1FBB1FEE1FFF1FA217B3076A
:107A1000E407F50720F0A21BB30BE40BF50B661F80
:107A2000771F881F991F1A9469F760957095809544
:107A300090959B01AC01BD01CF010895E199FECF66
:107A4000BFBBAEBBE09A11960DB20895E199FECF8F
:107A5000BFBBAEBB0DBA11960FB6F894E29AE19A8D
:067A60000FBE0895FFCFE8
:107A6600D60501009A016009E6005A009600F40165
:107A7600D0075401960050283C03190A64002C01D3
:107A860090011E00B00496001458022C01580214EE
:107A96000A0A0A179F023D00C01C41F401E203D7FF
:107AA60003C903B603A003840363033C030F03DE89
:107AB60002A902720239020002C901950164013865
:107AC600010F01EC00CC00B1009900840072006344
:107AD6000056004B004100390032002B00260022E0
:107AE600001E001A0017001500120064000000387E
:107AF60000380038003800380035003500350035CC
:107B0600003500010210080408102040802043615F
:107B16006C6962726174696E67004F323D002520A0
:107B260069643D0054673D002054773D00E2041B24
:107B36005B481B5B324A000D0A00202020202020D3
:107B46002020206F12833A0000803F004014544CDE
:107B5600616D6264610054657374004D52546563CF
:107B660068002020202020202020202020202020E7
:047B7600202020208B
:00000001FF
